******************************************************************************
            TI ARM Clang Linker PC v2.1.0                      
******************************************************************************
>> Linked Fri Nov 24 13:34:06 2023

OUTPUT FILE NAME:   <rfPacketTx_CC1312R1_LAUNCHXL_tirtos7_ticlang.out>
ENTRY POINT SYMBOL: "ResetISR"  address: 00008043


MEMORY CONFIGURATION

         name            origin    length      used     unused   attr    fill
----------------------  --------  ---------  --------  --------  ----  --------
  FLASH                 00000000   00058000  000090cf  0004ef31  R  X
  GPRAM                 11000000   00002000  00000000  00002000  RW X
  SRAM                  20000000   00014000  00005528  0000ead8  RW X
  LOG_DATA              90000000   00040000  00000000  00040000  R   


SEGMENT ALLOCATION MAP

run origin  load origin   length   init length attrs members
----------  ----------- ---------- ----------- ----- -------
00000000    00000000    00008f3b   00008f3b    r-x
  00000000    00000000    0000003c   0000003c    r-- .resetVecs
  0000003c    0000003c    0000808c   0000808c    r-x .text
  000080c8    000080c8    00000e73   00000e73    r-- .rodata
00008f3c    00008f3c    00000008   00000008    rw-
  00008f3c    00008f3c    00000008   00000008    rw- .args
00008f44    00008f44    00000134   00000134    r--
  00008f44    00008f44    00000134   00000134    r-- .cinit
00057fa8    00057fa8    00000058   00000058    r--
  00057fa8    00057fa8    00000058   00000058    r-- .ccfg
200000d8    200000d8    00004000   00000000    r--
  200000d8    200000d8    00004000   00000000    r-- .priheap
200040d8    200040d8    00001050   00000000    rw-
  200040d8    200040d8    00000aec   00000000    rw- .bss
  20004bc4    20004bc4    00000564   00000000    rw- .data
20013c00    20013c00    00000400   00000000    rw-
  20013c00    20013c00    00000400   00000000    rw- .stack


SECTION ALLOCATION MAP

 output                                  attributes/
section   page    origin      length       input sections
--------  ----  ----------  ----------   ----------------
.binit     0    00000000    00000000     

.cinit     0    00008f44    00000134     
                  00008f44    0000010d     (.cinit..data.load) [load image, compression = lzss]
                  00009051    00000003     --HOLE-- [fill = 0]
                  00009054    0000000c     (__TI_handler_table)
                  00009060    00000008     (.cinit..bss.load) [load image, compression = zero_init]
                  00009068    00000010     (__TI_cinit_table)

.init_array 
*          0    00000000    00000000     UNINITIALIZED

.ccfg      0    00057fa8    00000058     
                  00057fa8    00000058     ti_devices_config.o (.ccfg)

.bss       0    200040d8    00000aec     UNINITIALIZED
                  200040d8    000002c0     rf_multiMode_cc13x2.a : RFCC26X2_multiMode.c.cc13x2.ticlang.o (.bss.RF_cmdPool)
                  20004398    00000200     (.common:ti_sysbios_knl_Idle_taskStack)
                  20004598    00000100     rfPacketTx.o (.bss.rfObject)
                  20004698    000000d8     (.common:ti_sysbios_family_arm_m3_Hwi_dispatchTable)
                  20004770    0000007c     (.common:gpioCallbackFunctions)
                  200047ec    0000007c     (.common:gpioUserArgs)
                  20004868    00000068     rf_multiMode_cc13x2.a : RFCC26X2_multiMode.c.cc13x2.ticlang.o (.bss.RF_ratModule)
                  200048d0    00000060     (.common:ti_sysbios_knl_ClockSupport_timerStruct)
                  20004930    00000058     (.common:ti_sysbios_knl_Idle_taskStruct)
                  20004988    00000044                           : RFCC26X2_multiMode.c.cc13x2.ticlang.o (.bss.RF_clkInactivityObj)
                  200049cc    00000044                           : RFCC26X2_multiMode.c.cc13x2.ticlang.o (.bss.RF_clkPowerUpObj)
                  20004a10    0000003c                           : RFCC26X2_multiMode.c.cc13x2.ticlang.o (.bss.RF_swiHwObj)
                  20004a4c    00000030     (.common:ti_sysbios_knl_Swi_readyQs)
                  20004a7c    00000030     (.common:ti_sysbios_knl_Task_readyQs)
                  20004aac    0000002c     (.common:BIOS_heapMemObject)
                  20004ad8    00000028     (.common:BIOS_rtsGate)
                  20004b00    00000028     (.common:ti_sysbios_heaps_HeapMem_gate)
                  20004b28    00000020     (.common:ti_sysbios_runtime_System_atexitHandlers)
                  20004b48    0000001e     rfPacketTx.o (.bss.packet)
                  20004b66    00000002     --HOLE--
                  20004b68    0000001c     drivers_cc13x2.a : GPIOCC26X2.c.obj (.bss.gpioHwi)
                  20004b84    0000001c     ti_sysbios_config.o (.bss.sem)
                  20004ba0    00000004     driverlib.lib : osc.o (.bss.oscHfGlobals.0)
                  20004ba4    00000004                   : osc.o (.bss.oscHfGlobals.2)
                  20004ba8    00000004                   : osc.o (.bss.oscHfGlobals.3)
                  20004bac    00000004                   : osc.o (.bss.oscHfGlobals.4)
                  20004bb0    00000004     rfPacketTx.o (.bss.rfHandle)
                  20004bb4    00000004     (.common:PowerCC26XX_swiKey)
                  20004bb8    00000004     (.common:PowerCC26XX_taskKey)
                  20004bbc    00000004     (.common:ti_sysbios_family_arm_cc26xx_TimestampProvider_Module_state)
                  20004bc0    00000004     (.common:ti_sysbios_knl_Task_defaultStackHeap)

.data      0    20004bc4    00000564     UNINITIALIZED
                  20004bc4    00000174     drivers_cc13x2.a : PowerCC26X2.c.obj (.data.PowerCC26X2_module)
                  20004d38    0000007c     ti_drivers_config.o (.data.gpioPinConfigs)
                  20004db4    00000068     rf_multiMode_cc13x2.a : RFCC26X2_multiMode.c.cc13x2.ticlang.o (.data..L_MergedGlobals.1)
                  20004e1c    00000068     ti_sysbios_config.o (.data.ti_sysbios_knl_Clock_Module_state)
                  20004e84    00000064     rf_multiMode_cc13x2.a : RFCC26X2_multiMode.c.cc13x2.ticlang.o (.data..L_MergedGlobals.3)
                  20004ee8    00000058                           : RFCC26X2_multiMode.c.cc13x2.ticlang.o (.data..L_MergedGlobals.2)
                  20004f40    0000003c     ti_sysbios_config.o (.data.ti_sysbios_family_arm_m3_Hwi_Module_state)
                  20004f7c    0000003c     ti_sysbios_config.o (.data.ti_sysbios_knl_Task_Module_state)
                  20004fb8    0000002c     ti_sysbios_config.o (.data.BIOS_Module_state)
                  20004fe4    00000028     ti_radio_config.o (.data.RF_cmdPropRadioDivSetup)
                  2000500c    00000028     ti_radio_config.o (.data.pOverrides)
                  20005034    00000028     ti_sysbios_config.o (.data.ti_sysbios_knl_Swi_Module_state)
                  2000505c    00000018     ti_radio_config.o (.data.RF_cmdFs)
                  20005074    00000018     ti_radio_config.o (.data.RF_cmdPropTx)
                  2000508c    00000014     ti_sysbios_config.o (.data.defaultPthreadAttrs)
                  200050a0    00000010     ti_radio_config.o (.data.RF_prop)
                  200050b0    00000010     driverlib.lib : osc.o (.data._hposcCoeffs)
                  200050c0    0000000c     ti_sysbios_config.o (.data.ti_sysbios_family_arm_cc26xx_Timer_Module_state)
                  200050cc    0000000c     ti_sysbios_config.o (.data.ti_sysbios_runtime_Error_ignore)
                  200050d8    0000000c     ti_sysbios_config.o (.data.ti_sysbios_runtime_System_Module_state)
                  200050e4    00000008     rf_multiMode_cc13x2.a : RFCC26X2_multiMode.c.cc13x2.ticlang.o (.data..L_MergedGlobals)
                  200050ec    00000008                           : RFCC26X2_multiMode.c.cc13x2.ticlang.o (.data.RFCC26XX_schedulerPolicy)
                  200050f4    00000008     ti_sysbios_config.o (.data.ti_sysbios_gates_GateMutex_Module_state)
                  200050fc    00000008     ti_sysbios_config.o (.data.ti_sysbios_heaps_HeapMem_Module_state)
                  20005104    00000008     ti_sysbios_config.o (.data.ti_sysbios_knl_Semaphore_Module_state)
                  2000510c    00000004     rf_multiMode_cc13x2.a : RFCC26X2_multiMode.c.cc13x2.ticlang.o (.data.RF_fsmActiveState.lfClockSourceLast)
                  20005110    00000004     libc.a : aeabi_portable.c.obj (.data.__aeabi_errno)
                  20005114    00000004            : _lock.c.obj (.data._lock)
                  20005118    00000004            : _lock.c.obj (.data._unlock)
                  2000511c    00000004     ti_sysbios_config.o (.data.terminatedList)
                  20005120    00000004     ti_sysbios_config.o (.data.ti_sysbios_runtime_Memory_defaultHeapInstance)
                  20005124    00000001     rf_multiMode_cc13x2.a : rf_patch_cpe_prop.c.cc13x2.ticlang.o (.data.bPropPatchEntered)
                  20005125    00000001     drivers_cc13x2.a : GPIOCC26X2.c.obj (.data.initCalled)
                  20005126    00000001     ti_sysbios_config.o (.data.ti_sysbios_knl_Idle_initDone)
                  20005127    00000001     ti_sysbios_config.o (.data.ti_sysbios_runtime_Startup_done)

.stack     0    20013c00    00000400     UNINITIALIZED
                  20013c00    00000004     sysbios.a : boot_cortex_m.obj (.stack)
                  20013c04    000003fc     --HOLE--

.priheap   0    200000d8    00004000     UNINITIALIZED
                  200000d8    00004000     --HOLE--

.log_data 
*          0    90000000    00000000     COPY SECTION

.resetVecs 
*          0    00000000    0000003c     
                  00000000    0000003c     ti_sysbios_config.o (.resetVecs)

.vecs      0    20000000    000000d8     NOLOAD SECTION
                  20000000    000000d8     ti_sysbios_config.o (.vecs)

__llvm_prf_cnts 
*          0    20000000    00000000     UNINITIALIZED

__llvm_prf_bits 
*          0    20000000    00000000     UNINITIALIZED

.text      0    0000003c    0000808c     
                  0000003c    00000498     rf_multiMode_cc13x2.a : RFCC26X2_multiMode.c.cc13x2.ticlang.o (.text.RF_fsmActiveState)
                  000004d4    0000029c                           : RFCC26X2_multiMode.c.cc13x2.ticlang.o (.text.RF_open)
                  00000770    000001fa     ti_sysbios_config.o (.text.ti_sysbios_family_arm_m3_Hwi_excFillContext)
                  0000096a    00000002     ti_sysbios_config.o (.text.BIOS_nullFunc)
                  0000096c    000001e0     rf_multiMode_cc13x2.a : RFCC26X2_multiMode.c.cc13x2.ticlang.o (.text.RF_dispatchNextCmd)
                  00000b4c    000001b2     rfPacketTx.o (.text.mainThread)
                  00000cfe    000001aa     ti_sysbios_config.o (.text.ti_sysbios_knl_TaskSupport_buildTaskStack)
                  00000ea8    00000198     ti_sysbios_config.o (.text.ti_sysbios_family_arm_cc26xx_Timer_construct)
                  00001040    00000194     drivers_cc13x2.a : PowerCC26X2_calibrateRCOSC.c.obj (.text.PowerCC26X2_auxISR)
                  000011d4    0000018e     ti_sysbios_config.o (.text.ti_sysbios_knl_Task_Instance_init)
                  00001362    00000002     ti_drivers_config.o (.text.Board_initHook)
                  00001364    0000015c     drivers_cc13x2.a : PowerCC26X2.c.obj (.text.Power_sleep)
                  000014c0    0000014e     ti_sysbios_config.o (.text.pthread_create)
                  0000160e    0000013e     ti_sysbios_config.o (.text.PowerCC26XX_standbyPolicy)
                  0000174c    0000013e     ti_sysbios_config.o (.text.ti_sysbios_heaps_HeapMem_allocUnprotected)
                  0000188a    00000002     rf_multiMode_cc13x2.a : rfc.c.cc13x2.ticlang.o (.text.NOROM_RFCCpePatchReset)
                  0000188c    0000013c                           : RFCC26X2_multiMode.c.cc13x2.ticlang.o (.text.RF_radioOpDoneCb)
                  000019c8    0000013c     ti_sysbios_config.o (.text.ti_sysbios_knl_Clock_workFuncDynamic)
                  00001b04    00000134     ti_sysbios_config.o (.text.ti_sysbios_knl_Task_setPri)
                  00001c38    0000012c     rf_multiMode_cc13x2.a : RFCC26X2_multiMode.c.cc13x2.ticlang.o (.text.RF_fsmSetupState)
                  00001d64    00000124                           : RFCC26X2_multiMode.c.cc13x2.ticlang.o (.text.RF_abortCmd)
                  00001e88    0000011c     sysbios.a : Hwi_asm_gnu.obj (.text.ti_sysbios_family_arm_m3_Hwi_dispatch)
                  00001fa4    00000118     drivers_cc13x2.a : PowerCC26X2.c.obj (.text.Power_init)
                  000020bc    00000118     rf_multiMode_cc13x2.a : RFCC26X2_multiMode.c.cc13x2.ticlang.o (.text.RF_decodeOverridePointers)
                  000021d4    0000010e     ti_sysbios_config.o (.text.ti_sysbios_knl_Semaphore_pend)
                  000022e2    00000002     rf_multiMode_cc13x2.a : RFCC26X2_multiMode.c.cc13x2.ticlang.o (.text.RF_defaultCallback)
                  000022e4    0000010c     drivers_cc13x2.a : PowerCC26X2_calibrateRCOSC.c.obj (.text.PowerCC26X2_calibrate)
                  000023f0    0000010a     ti_sysbios_config.o (.text.ti_sysbios_knl_Task_Instance_finalize)
                  000024fa    00000002     libclang_rt.builtins.a : aeabi_div0.c.obj (.text.__aeabi_ldiv0)
                  000024fc    00000108     rf_multiMode_cc13x2.a : RFCC26X2_multiMode.c.cc13x2.ticlang.o (.text.RF_fsmPowerUpState)
                  00002604    00000104     drivers_cc13x2.a : GPIOCC26X2.c.obj (.text.GPIO_init)
                  00002708    000000fe     ti_sysbios_config.o (.text.ti_sysbios_family_arm_m3_Hwi_Instance_init)
                  00002806    00000002     libc.a : _lock.c.obj (.text._nop)
                  00002808    000000fc     rf_multiMode_cc13x2.a : RFCC26X2_multiMode.c.cc13x2.ticlang.o (.text.RF_hwiCpe0Active)
                  00002904    000000f4     driverlib.lib : sys_ctrl.o (.text.NOROM_SysCtrlStandby)
                  000029f8    000000ee     ti_sysbios_config.o (.text.ti_sysbios_knl_Clock_startI)
                  00002ae6    000000e4     ti_sysbios_config.o (.text.ti_sysbios_family_arm_m3_Hwi_initNVIC)
                  00002bca    000000dc     ti_sysbios_config.o (.text.ti_sysbios_knl_Task_checkStacks)
                  00002ca6    000000da     ti_sysbios_config.o (.text.ti_sysbios_heaps_HeapMem_freeUnprotected)
                  00002d80    000000d0     drivers_cc13x2.a : PowerCC26X2.c.obj (.text.configureXOSCHF)
                  00002e50    000000cc     rf_multiMode_cc13x2.a : RFCC26X2_multiMode.c.cc13x2.ticlang.o (.text.RF_postCmd)
                  00002f1c    000000ca                           : RFCC26X2_multiMode.c.cc13x2.ticlang.o (.text.RF_updatePaConfiguration)
                  00002fe6    000000ca     ti_sysbios_config.o (.text._pthread_removeThreadKeys)
                  000030b0    000000c4     driverlib.lib : setup.o (.text.NOROM_SetupTrimDevice)
                  00003174    000000c4                   : setup.o (.text.TrimAfterColdResetWakeupFromShutDown)
                  00003238    000000c0     ti_sysbios_config.o (.text.ti_sysbios_knl_Clock_walkQueueDynamic)
                  000032f8    000000c0     ti_sysbios_config.o (.text.ti_sysbios_knl_Swi_restoreHwi)
                  000033b8    000000bc     rf_multiMode_cc13x2.a : RFCC26X2_multiMode.c.cc13x2.ticlang.o (.text.RF_swiHw)
                  00003474    000000bc     ti_sysbios_config.o (.text.ti_sysbios_knl_Task_postInit)
                  00003530    000000b8     ti_sysbios_config.o (.text.ti_sysbios_knl_Swi_Instance_init)
                  000035e8    000000b4     driverlib.lib : osc.o (.text.NOROM_OSCHF_AttemptToSwitchToXosc)
                  0000369c    000000b4     drivers_cc13x2.a : PowerCC26X2.c.obj (.text.Power_releaseDependency)
                  00003750    000000b0                      : PowerCC26X2.c.obj (.text.Power_setDependency)
                  00003800    000000b0     libclang_rt.builtins.a : udivmoddi4.S.obj (.text)
                  000038b0    000000ac     rf_multiMode_cc13x2.a : RFCC26X2_multiMode.c.cc13x2.ticlang.o (.text.RF_initRadioSetup)
                  0000395c    000000ac                           : RFCC26X2_multiMode.c.cc13x2.ticlang.o (.text.RF_pendCmd)
                  00003a08    000000aa     driverlib.lib : chipinfo.o (.text.NOROM_ChipInfo_GetChipType)
                  00003ab2    000000a2     ti_sysbios_config.o (.text.ti_sysbios_knl_TaskSupport_start)
                  00003b54    000000a2     ti_sysbios_config.o (.text.ti_sysbios_knl_Task_schedule)
                  00003bf6    00000002     drivers_cc13x2.a : PowerCC26X2.c.obj (.text.emptyClockFunc)
                  00003bf8    000000a0     rf_multiMode_cc13x2.a : RFCC26X2_multiMode.c.cc13x2.ticlang.o (.text.RF_calculateDispatchTime)
                  00003c98    0000009a                           : RFCC26X2_multiMode.c.cc13x2.ticlang.o (.text.RF_defaultSubmitPolicy)
                  00003d32    00000096                           : RFCC26X2_multiMode.c.cc13x2.ticlang.o (.text.RF_verifyGap)
                  00003dc8    00000094                           : RFCC26X2_multiMode.c.cc13x2.ticlang.o (.text.RF_ratRestartChannels)
                  00003e5c    00000094     ti_sysbios_config.o (.text.ti_sysbios_heaps_HeapMem_Instance_init)
                  00003ef0    00000090     ti_sysbios_config.o (.text.ti_sysbios_knl_Task_sleep)
                  00003f80    0000008e     ti_sysbios_config.o (.text.ti_sysbios_family_arm_m3_Hwi_excHandlerMin)
                  0000400e    0000008e     ti_sysbios_config.o (.text.ti_sysbios_knl_Swi_runLoop)
                  0000409c    0000008c     drivers_cc13x2.a : GPIOCC26XX.c.obj (.text.GPIO_setConfig)
                  00004128    0000008c     ti_sysbios_config.o (.text.ti_sysbios_family_arm_m3_Hwi_construct2)
                  000041b4    0000008a     ti_sysbios_config.o (.text.ti_sysbios_knl_Semaphore_post)
                  0000423e    00000002     ti_sysbios_config.o (.text.ti_sysbios_family_arm_cc26xx_Timer_startup)
                  00004240    00000088     rf_multiMode_cc13x2.a : RFCC26X2_multiMode.c.cc13x2.ticlang.o (.text.RF_cmdDispatchTime)
                  000042c8    00000088                           : RFCC26X2_multiMode.c.cc13x2.ticlang.o (.text.RF_discardPendCmd)
                  00004350    00000088     ti_sysbios_config.o (.text.ti_sysbios_family_arm_m3_Hwi_postInit)
                  000043d8    00000086     ti_sysbios_config.o (.text.ti_sysbios_runtime_Memory_alloc)
                  0000445e    00000002     ti_sysbios_config.o (.text.ti_sysbios_knl_TaskSupport_init)
                  00004460    00000084     rf_multiMode_cc13x2.a : RFCC26X2_multiMode.c.cc13x2.ticlang.o (.text.RF_yield)
                  000044e4    00000084     ti_sysbios_config.o (.text.ti_sysbios_knl_Task_startup)
                  00004568    00000082     ti_sysbios_config.o (.text.ti_sysbios_family_arm_m3_Hwi_getStackInfo)
                  000045ea    00000080     driverlib.lib : sys_ctrl.o (.text.NOROM_SysCtrlSetRechargeBeforePowerDown)
                  0000466a    00000080     main_tirtos.o (.text.main)
                  000046ea    0000007e     ti_drivers_config.o (.text.Board_sendExtFlashByte)
                  00004768    0000007c     ti_sysbios_config.o (.text.SwiP_construct)
                  000047e4    0000007c     ti_sysbios_config.o (.text.pthread_exit)
                  00004860    0000007c     ti_sysbios_config.o (.text.ti_sysbios_family_arm_cc26xx_Timer_periodicStub)
                  000048dc    0000007c     ti_sysbios_config.o (.text.ti_sysbios_knl_Swi_schedule)
                  00004958    0000007a     ti_sysbios_config.o (.text.ti_sysbios_family_arm_m3_Hwi_dispatchC)
                  000049d2    0000007a     ti_sysbios_config.o (.text.ti_sysbios_knl_Idle_init)
                  00004a4c    00000078     driverlib.lib : osc.o (.text.NOROM_OSCHF_SwitchToRcOscTurnOffXosc)
                  00004ac4    00000078                   : osc.o (.text.NOROM_OSC_CapArrayAdjustWorkaround_Boot)
                  00004b3c    00000078     drivers_cc13x2.a : PowerCC26X2_calibrateRCOSC_helpers.c.obj (.text.PowerCC26X2_updateSubSecInc)
                  00004bb4    00000078     rf_multiMode_cc13x2.a : RFCC26X2_multiMode.c.cc13x2.ticlang.o (.text.RF_ratFreeChannel)
                  00004c2c    00000078     ti_sysbios_config.o (.text.ti_sysbios_family_arm_m3_Hwi_disableInterrupt)
                  00004ca4    00000078     ti_sysbios_config.o (.text.ti_sysbios_knl_Swi_run)
                  00004d1c    00000078     ti_sysbios_config.o (.text.ti_sysbios_knl_Task_blockI)
                  00004d94    00000074     rf_multiMode_cc13x2.a : RFCC26X2_multiMode.c.cc13x2.ticlang.o (.text.RF_hwiHw)
                  00004e08    00000074     ti_sysbios_config.o (.text.ti_sysbios_heaps_HeapMem_getStats)
                  00004e7c    00000072     ti_sysbios_config.o (.text.ti_sysbios_family_arm_cc26xx_Timer_setThreshold)
                  00004eee    00000070     ti_sysbios_config.o (.text.ti_sysbios_family_arm_m3_Hwi_enableInterrupt)
                  00004f5e    0000006e     ti_sysbios_config.o (.text.BIOS_init)
                  00004fcc    0000006e     ti_drivers_config.o (.text.Board_shutDownExtFlash)
                  0000503a    0000006e     ti_sysbios_config.o (.text.ti_sysbios_knl_Clock_init)
                  000050a8    0000006c     rf_multiMode_cc13x2.a : RFCC26X2_multiMode.c.cc13x2.ticlang.o (.text.RF_issueRadioFreeCb)
                  00005114    0000006a                           : RFCC26X2_multiMode.c.cc13x2.ticlang.o (.text.RF_detachOverrides)
                  0000517e    0000006a     libc.a : copy_decompress_lzss.c.obj (.text:decompress:lzss)
                  000051e8    00000066     rf_multiMode_cc13x2.a : RFCC26X2_multiMode.c.cc13x2.ticlang.o (.text.RF_attachOverrides)
                  0000524e    00000066     ti_sysbios_config.o (.text.ti_sysbios_family_arm_cc26xx_Timer_start)
                  000052b4    00000066     ti_sysbios_config.o (.text.ti_sysbios_family_arm_m3_Hwi_Instance_finalize)
                  0000531a    00000002     ti_sysbios_config.o (.text.ti_sysbios_runtime_SysCallback_defaultInit)
                  0000531c    00000064     drivers_cc13x2.a : PowerCC26X2_calibrateRCOSC.c.obj (.text.PowerCC26X2_initiateCalibration)
                  00005380    00000064     rf_multiMode_cc13x2.a : RFCC26X2_multiMode.c.cc13x2.ticlang.o (.text.RF_dispatchNextEvent)
                  000053e4    00000064                           : RFCC26X2_multiMode.c.cc13x2.ticlang.o (.text.RF_hwiCpe0PowerFsm)
                  00005448    00000062                           : RFCC26X2_multiMode.c.cc13x2.ticlang.o (.text.RF_syncCb)
                  000054aa    00000060     ti_sysbios_config.o (.text.ti_sysbios_knl_ClockSupport_init)
                  0000550a    00000002     --HOLE-- [fill = 0]
                  0000550c    0000005e     rf_multiMode_cc13x2.a : rfc.c.cc13x2.ticlang.o (.text.NOROM_RFCAnaDivTxOverride)
                  0000556a    0000005e     ti_sysbios_config.o (.text.ti_sysbios_knl_Swi_post)
                  000055c8    0000005c     ti_sysbios_config.o (.text.ClockP_construct)
                  00005624    0000005c     ti_sysbios_config.o (.text.ti_sysbios_heaps_HeapMem_alloc)
                  00005680    0000005c     ti_sysbios_config.o (.text.ti_sysbios_knl_Task_init)
                  000056dc    00000058     ti_sysbios_config.o (.text.AONRTCEventClear)
                  00005734    00000058     ti_sysbios_config.o (.text.HwiP_construct)
                  0000578c    00000058     rf_multiMode_cc13x2.a : RFCC26X2_multiMode.c.cc13x2.ticlang.o (.text.RF_applyRfCorePatch)
                  000057e4    00000058     ti_sysbios_config.o (.text.ti_sysbios_family_arm_m3_Hwi_construct)
                  0000583c    00000058     sysbios.a : Hwi_asm_switch_gnu.obj (.text.ti_sysbios_family_arm_m3_Hwi_initStacks)
                  00005894    00000058     ti_sysbios_config.o (.text.ti_sysbios_heaps_HeapMem_construct)
                  000058ec    00000058     ti_sysbios_config.o (.text.ti_sysbios_knl_Swi_init)
                  00005944    00000056     ti_sysbios_config.o (.text.AONRTCCompareValueSet)
                  0000599a    00000056     ti_sysbios_config.o (.text.ti_sysbios_family_arm_cc26xx_Timer_getCurrentTick)
                  000059f0    00000056     ti_sysbios_config.o (.text.ti_sysbios_knl_Clock_Instance_init)
                  00005a46    00000056     ti_sysbios_config.o (.text.ti_sysbios_runtime_System_atexit)
                  00005a9c    00000054     ti_sysbios_config.o (.text.AONRTCChannelEnable)
                  00005af0    00000054     ti_sysbios_config.o (.text.BIOS_startFunc)
                  00005b44    00000054     rf_multiMode_cc13x2.a : RFCC26X2_multiMode.c.cc13x2.ticlang.o (.text.RF_fsmXOSCState)
                  00005b98    00000054                           : RFCC26X2_multiMode.c.cc13x2.ticlang.o (.text.RF_getCurrentTime)
                  00005bec    00000054     ti_sysbios_config.o (.text.pthread_setcancelstate)
                  00005c40    00000052     driverlib.lib : chipinfo.o (.text.NOROM_ChipInfo_GetHwRevision)
                  00005c92    00000052     ti_sysbios_config.o (.text.usleep)
                  00005ce4    00000050     rf_multiMode_cc13x2.a : RFCC26X2_multiMode.c.cc13x2.ticlang.o (.text.RF_wakeupNotification)
                  00005d34    00000050     ti_sysbios_config.o (.text.ti_sysbios_family_arm_cc26xx_Timer_setNextTick)
                  00005d84    0000004e     ti_sysbios_config.o (.text.ti_sysbios_knl_Swi_restore)
                  00005dd2    0000004c     driverlib.lib : osc.o (.text.NOROM_OSC_HPOSCRelativeFrequencyOffsetGet)
                  00005e1e    00000002     --HOLE-- [fill = 0]
                  00005e20    0000004c     drivers_cc13x2.a : PowerCC26X2.c.obj (.text.switchXOSCHF)
                  00005e6c    0000004c     ti_sysbios_config.o (.text.ti_sysbios_knl_Clock_getTimeout)
                  00005eb8    0000004c     ti_sysbios_config.o (.text.ti_sysbios_knl_Task_create)
                  00005f04    0000004c     ti_sysbios_config.o (.text.ti_sysbios_runtime_System_processAtExit)
                  00005f50    0000004a     ti_sysbios_config.o (.text.ti_sysbios_knl_Task_construct)
                  00005f9a    00000002     --HOLE-- [fill = 0]
                  00005f9c    00000048     driverlib.lib : aux_sysif.o (.text.NOROM_AUXSYSIFOpModeChange)
                  00005fe4    00000048     rf_multiMode_cc13x2.a : rfc.c.cc13x2.ticlang.o (.text.NOROM_RFCSynthPowerDown)
                  0000602c    00000048     drivers_cc13x2.a : PowerCC26X2.c.obj (.text.PowerCC26XX_switchXOSC_HF)
                  00006074    00000048                      : PowerCC26X2.c.obj (.text.oscillatorISR)
                  000060bc    00000048     ti_sysbios_config.o (.text.ti_sysbios_family_arm_m3_Hwi_init)
                  00006104    00000046     ti_sysbios_config.o (.text.ti_sysbios_knl_Semaphore_Instance_init)
                  0000614a    00000046     ti_sysbios_config.o (.text.ti_sysbios_knl_Swi_construct)
                  00006190    00000046     ti_sysbios_config.o (.text.ti_sysbios_knl_Task_processVitalTaskFlag)
                  000061d6    00000046     ti_sysbios_config.o (.text.ti_sysbios_knl_Task_unblockI)
                  0000621c    00000044     ti_sysbios_config.o (.text.BIOS_rtsLock)
                  00006260    00000044     drivers_cc13x2.a : GPIOCC26X2.c.obj (.text.GPIO_hwiIntFxn)
                  000062a4    00000044     driverlib.lib : prcm.o (.text.NOROM_PRCMPowerDomainsAllOff)
                  000062e8    00000044                   : prcm.o (.text.NOROM_PRCMPowerDomainsAllOn)
                  0000632c    00000044     drivers_cc13x2.a : PowerCC26X2.c.obj (.text.PowerCC26XX_isStableXOSC_HF)
                  00006370    00000044     rf_multiMode_cc13x2.a : RFCC26X2_multiMode.c.cc13x2.ticlang.o (.text.RF_cmdGet)
                  000063b4    00000044                           : RFCC26X2_multiMode.c.cc13x2.ticlang.o (.text.RF_updatePowerupDuration)
                  000063f8    00000044     ti_sysbios_config.o (.text._pthread_cleanupFxn)
                  0000643c    00000044     ti_sysbios_config.o (.text.ti_sysbios_knl_Task_restore)
                  00006480    00000044     ti_sysbios_config.o (.text.ti_sysbios_runtime_Error_raiseX)
                  000064c4    00000040     drivers_cc13x2.a : PowerCC26X2_calibrateRCOSC.c.obj (.text.PowerCC26X2_RCOSC_clockFunc)
                  00006504    00000040                      : PowerCC26X2_calibrateRCOSC_helpers.c.obj (.text.PowerCC26X2_setAclkRefSrc)
                  00006544    00000040     ti_sysbios_config.o (.text.ti_sysbios_gates_GateMutex_enter)
                  00006584    00000040     ti_sysbios_config.o (.text.ti_sysbios_knl_Semaphore_pendTimeout)
                  000065c4    00000040     ti_sysbios_config.o (.text.ti_sysbios_knl_Task_exit)
                  00006604    0000003e     ti_sysbios_config.o (.text.pthread_attr_setschedparam)
                  00006642    0000003e     ti_sysbios_config.o (.text.ti_sysbios_knl_Clock_getTicksUntilInterrupt)
                  00006680    0000003c     ti_sysbios_config.o (.text.BIOS_atExitFunc)
                  000066bc    0000003c     drivers_cc13x2.a : GPIO.c.obj (.text.GPIO_resetConfig)
                  000066f8    0000003c     driverlib.lib : sys_ctrl.o (.text.NOROM_SysCtrlIdle)
                  00006734    0000003c     drivers_cc13x2.a : PowerCC26X2_calibrateRCOSC_helpers.c.obj (.text.PowerCC26X2_setTdcClkSrc24M)
                  00006770    0000003c     ti_sysbios_config.o (.text.ti_sysbios_family_arm_m3_Hwi_setPriority)
                  000067ac    0000003c     ti_sysbios_config.o (.text.ti_sysbios_knl_Task_restoreHwi)
                  000067e8    00000038     ti_drivers_config.o (.text.Board_wakeUpExtFlash)
                  00006820    00000038     drivers_cc13x2.a : PowerCC26X2_helpers.c.obj (.text.PowerCC26X2_oscDisableQualifiers)
                  00006858    00000038     rf_multiMode_cc13x2.a : rf_patch_cpe_prop.c.cc13x2.ticlang.o (.text.configurePropPatch)
                  00006890    00000038     ti_sysbios_config.o (.text.ti_sysbios_runtime_Startup_exec)
                  000068c8    00000038     libc.a : autoinit.c.obj (.text:__TI_auto_init_nobinit_nopinit)
                  00006900    00000036     ti_sysbios_config.o (.text.BIOS_rtsUnlock)
                  00006936    00000036     ti_sysbios_config.o (.text.SemaphoreP_pend)
                  0000696c    00000036     ti_sysbios_config.o (.text.ti_sysbios_knl_Swi_construct2)
                  000069a2    00000002     --HOLE-- [fill = 0]
                  000069a4    00000034     drivers_cc13x2.a : PowerCC26X2.c.obj (.text.Power_releaseConstraint)
                  000069d8    00000034     rf_multiMode_cc13x2.a : RFCC26X2_multiMode.c.cc13x2.ticlang.o (.text.RF_powerConstraintRelease)
                  00006a0c    00000034     ti_sysbios_config.o (.text.ti_sysbios_family_arm_cc26xx_Timer_getMaxTicks)
                  00006a40    00000034     ti_sysbios_config.o (.text.ti_sysbios_knl_Queue_put)
                  00006a74    00000034     sysbios.a : boot_cortex_m.obj (.text:_c_int00)
                  00006aa8    00000030     drivers_cc13x2.a : PowerCC26X2.c.obj (.text.Power_setConstraint)
                  00006ad8    00000030     rf_multiMode_cc13x2.a : RFCC26X2_multiMode.c.cc13x2.ticlang.o (.text.RF_checkCmdFsError)
                  00006b08    00000030     drivers_cc13x2.a : PowerCC26X2.c.obj (.text.notify)
                  00006b38    00000030     ti_sysbios_config.o (.text.ti_sysbios_family_arm_m3_Hwi_plug)
                  00006b68    00000030     ti_sysbios_config.o (.text.ti_sysbios_heaps_HeapMem_free)
                  00006b98    00000030     ti_sysbios_config.o (.text.ti_sysbios_knl_Clock_construct)
                  00006bc8    00000030     ti_sysbios_config.o (.text.ti_sysbios_knl_Idle_run)
                  00006bf8    0000002e     driverlib.lib : chipinfo.o (.text.NOROM_ThisLibraryIsFor_CC13x2_CC26x2_HwRev20AndLater_HaltIfViolated)
                  00006c26    0000002e     rf_multiMode_cc13x2.a : RFCC26X2_multiMode.c.cc13x2.ticlang.o (.text.RF_calculateDeltaTimeUs)
                  00006c54    0000002e     ti_sysbios_config.o (.text._pthread_delete)
                  00006c82    0000002e     ti_sysbios_config.o (.text._pthread_runStub)
                  00006cb0    0000002e     ti_sysbios_config.o (.text.ti_sysbios_family_arm_m3_Hwi_initStack)
                  00006cde    0000002e     ti_sysbios_config.o (.text.ti_sysbios_gates_GateMutex_Instance_init)
                  00006d0c    0000002c     ti_sysbios_config.o (.text.BIOS_registerRTSLock)
                  00006d38    0000002c     ti_sysbios_config.o (.text.BIOS_removeRTSLock)
                  00006d64    0000002c     rf_multiMode_cc13x2.a : RFCC26X2_multiMode.c.cc13x2.ticlang.o (.text.RF_executeDirectImmediateCmd)
                  00006d90    0000002c     ti_sysbios_config.o (.text.pthread_attr_setdetachstate)
                  00006dbc    0000002c     rf_multiMode_cc13x2.a : rf_patch_cpe_prop.c.cc13x2.ticlang.o (.text.rf_patch_cpe_prop)
                  00006de8    0000002c     ti_sysbios_config.o (.text.ti_sysbios_knl_Semaphore_construct)
                  00006e14    0000002c     ti_sysbios_config.o (.text.ti_sysbios_runtime_Memory_free)
                  00006e40    0000002a     driverlib.lib : osc.o (.text.NOROM_OSCHF_TurnOnXosc)
                  00006e6a    0000002a     ti_sysbios_config.o (.text.SemaphoreP_constructBinary)
                  00006e94    0000002a     ti_sysbios_config.o (.text._pthread_cleanup_pop)
                  00006ebe    0000002a     ti_sysbios_config.o (.text.pthread_attr_init)
                  00006ee8    0000002a     ti_sysbios_config.o (.text.ti_sysbios_knl_Clock_initI)
                  00006f12    0000002a     ti_sysbios_config.o (.text.ti_sysbios_knl_Task_enter)
                  00006f3c    00000028     drivers_cc13x2.a : List.c.obj (.text.List_remove)
                  00006f64    00000028     rf_multiMode_cc13x2.a : RFCC26X2_multiMode.c.cc13x2.ticlang.o (.text.RF_cmdStoreEvents)
                  00006f8c    00000028     sysbios.a : Hwi_asm_gnu.obj (.text.ti_sysbios_family_arm_m3_Hwi_excHandlerAsm)
                  00006fb4    00000028     ti_sysbios_config.o (.text.ti_sysbios_gates_GateMutex_construct)
                  00006fdc    00000028     ti_sysbios_config.o (.text.ti_sysbios_knl_Queue_enqueue)
                  00007004    00000028     ti_sysbios_config.o (.text.ti_sysbios_knl_Queue_insert)
                  0000702c    00000028     ti_sysbios_config.o (.text.ti_sysbios_knl_Swi_or)
                  00007054    00000028     ti_sysbios_config.o (.text.ti_sysbios_knl_TaskSupport_checkStack)
                  0000707c    00000028     sysbios.a : TaskSupport_asm_gnu.obj (.text.ti_sysbios_knl_TaskSupport_swap)
                  000070a4    00000028     ti_sysbios_config.o (.text.ti_sysbios_knl_Task_sleepTimeout)
                  000070cc    00000028     ti_sysbios_config.o (.text.ti_sysbios_runtime_System_init)
                  000070f4    00000026     drivers_cc13x2.a : List.c.obj (.text.List_insert)
                  0000711a    00000026                      : List.c.obj (.text.List_putHead)
                  00007140    00000026     rf_multiMode_cc13x2.a : RFCC26X2_multiMode.c.cc13x2.ticlang.o (.text.RF_runCmd)
                  00007166    00000026     ti_sysbios_config.o (.text.ti_sysbios_family_arm_m3_Hwi_getHandle)
                  0000718c    00000026     ti_sysbios_config.o (.text.ti_sysbios_knl_Task_allBlockedFunction)
                  000071b2    00000026     ti_sysbios_config.o (.text.ti_sysbios_knl_Task_delete)
                  000071d8    00000026     ti_sysbios_config.o (.text.ti_sysbios_knl_Task_destruct)
                  000071fe    00000026     ti_sysbios_config.o (.text.ti_sysbios_runtime_Error_init)
                  00007224    00000024     ti_sysbios_config.o (.text.HwiP_setFunc)
                  00007248    00000024     drivers_cc13x2.a : List.c.obj (.text.List_put)
                  0000726c    00000024                      : PowerCC26X2_calibrateRCOSC_helpers.c.obj (.text.PowerCC26X2_writeCtrim)
                  00007290    00000024                      : PowerCC26X2_calibrateRCOSC_helpers.c.obj (.text.PowerCC26X2_writeCtrimFract)
                  000072b4    00000024                      : PowerCC26X2_calibrateRCOSC_helpers.c.obj (.text.PowerCC26X2_writeCtrimFractEn)
                  000072d8    00000024                      : PowerCC26X2_calibrateRCOSC_helpers.c.obj (.text.PowerCC26X2_writeRtrim)
                  000072fc    00000024                      : PowerCC26X2.c.obj (.text.Power_registerNotify)
                  00007320    00000024     rf_multiMode_cc13x2.a : RFCC26X2_multiMode.c.cc13x2.ticlang.o (.text.RF_clkPowerUp)
                  00007344    00000024                           : RFCC26X2_multiMode.c.cc13x2.ticlang.o (.text.RF_hwiCpe0ChangePhy)
                  00007368    00000024                           : RFCC26X2_multiMode.c.cc13x2.ticlang.o (.text.RF_isStateTransitionAllowed)
                  0000738c    00000024                           : RFCC26X2_multiMode.c.cc13x2.ticlang.o (.text.RF_searchAndReplacePAOverride)
                  000073b0    00000024     ti_sysbios_config.o (.text.ti_sysbios_family_arm_cc26xx_Timer_Params_init)
                  000073d4    00000024     ti_sysbios_config.o (.text.ti_sysbios_knl_Task_Params_init)
                  000073f8    00000022     ti_sysbios_config.o (.text.BIOS_setThreadType)
                  0000741a    00000022     drivers_cc13x2.a : List.c.obj (.text.List_get)
                  0000743c    00000022     ti_sysbios_config.o (.text.ti_sysbios_gates_GateMutex_leave)
                  0000745e    00000022     ti_sysbios_config.o (.text.ti_sysbios_heaps_HeapMem_restore)
                  00007480    00000022     ti_sysbios_config.o (.text.ti_sysbios_knl_Clock_getTicks)
                  000074a2    00000022     ti_sysbios_config.o (.text.ti_sysbios_knl_Clock_scheduleNextTick)
                  000074c4    00000022     ti_sysbios_config.o (.text.ti_sysbios_knl_Queue_dequeue)
                  000074e6    00000022     ti_sysbios_config.o (.text.ti_sysbios_knl_Semaphore_destruct)
                  00007508    00000020     rf_multiMode_cc13x2.a : rfc.c.cc13x2.ticlang.o (.text.NOROM_RFCDoorbellSendTo)
                  00007528    00000020                           : rfc.c.cc13x2.ticlang.o (.text.NOROM_RFCOverrideSearch)
                  00007548    00000020     drivers_cc13x2.a : PowerCC26X2_helpers.c.obj (.text.PowerCC26X2_disableTCXOQual)
                  00007568    00000020                      : PowerCC26X2_helpers.c.obj (.text.PowerCC26X2_enableTCXOQual)
                  00007588    00000020     ti_sysbios_config.o (.text.PowerCC26XX_schedulerDisable)
                  000075a8    00000020     ti_sysbios_config.o (.text.PowerCC26XX_schedulerRestore)
                  000075c8    00000020     rf_multiMode_cc13x2.a : RFCC26X2_multiMode.c.cc13x2.ticlang.o (.text.RF_cmdAlloc)
                  000075e8    00000020                           : RFCC26X2_multiMode.c.cc13x2.ticlang.o (.text.RF_invokeGlobalCallback)
                  00007608    00000020                           : RFCC26X2_multiMode.c.cc13x2.ticlang.o (.text.RF_ratIsRunning)
                  00007628    00000020     ti_sysbios_config.o (.text.ti_sysbios_family_arm_cc26xx_Timer_postInit)
                  00007648    00000020     ti_sysbios_config.o (.text.ti_sysbios_family_arm_m3_Hwi_excHandler)
                  00007668    00000020     ti_sysbios_config.o (.text.ti_sysbios_family_arm_m3_Hwi_post)
                  00007688    00000020     ti_sysbios_config.o (.text.ti_sysbios_knl_ClockSupport_getCurrentTick)
                  000076a8    0000001e     ti_sysbios_config.o (.text.SwiP_Params_init)
                  000076c6    0000001e     sysbios.a : Hwi_asm_switch_gnu.obj (.text.ti_sysbios_family_arm_m3_Hwi_switchAndRunFunc)
                  000076e4    0000001e     ti_sysbios_config.o (.text.ti_sysbios_family_arm_m3_Hwi_switchFromBootStack)
                  00007702    0000001e     ti_sysbios_config.o (.text.ti_sysbios_knl_Task_unblock)
                  00007720    0000001c     ti_sysbios_config.o (.text.HwiP_Params_init)
                  0000773c    0000001c     drivers_cc13x2.a : PowerCC26X2.c.obj (.text.Power_getTransitionLatency)
                  00007758    0000001c     rf_multiMode_cc13x2.a : RFCC26X2_multiMode.c.cc13x2.ticlang.o (.text.RF_clkInactivityCallback)
                  00007774    0000001c                           : RFCC26X2_multiMode.c.cc13x2.ticlang.o (.text.RF_getPAOverrideOffsetAndValue)
                  00007790    0000001c                           : RFCC26X2_multiMode.c.cc13x2.ticlang.o (.text.RF_powerConstraintSet)
                  000077ac    0000001c                           : RFCC26X2_multiMode.c.cc13x2.ticlang.o (.text.RF_swiFsm)
                  000077c8    0000001c     ti_sysbios_config.o (.text.ti_sysbios_family_arm_cc26xx_Timer_dynamicStub)
                  000077e4    0000001c     ti_sysbios_config.o (.text.ti_sysbios_family_arm_m3_Hwi_Params_init)
                  00007800    0000001c     ti_sysbios_config.o (.text.ti_sysbios_knl_Clock_enqueueI)
                  0000781c    0000001c     ti_sysbios_config.o (.text.ti_sysbios_knl_Clock_start)
                  00007838    0000001c     ti_sysbios_config.o (.text.ti_sysbios_knl_Queue_remove)
                  00007854    0000001c     ti_sysbios_config.o (.text.ti_sysbios_knl_Swi_Params_init)
                  00007870    0000001c     ti_sysbios_config.o (.text.ti_sysbios_knl_Swi_disable)
                  0000788c    0000001c     ti_sysbios_config.o (.text.ti_sysbios_knl_Task_disable)
                  000078a8    0000001a     ti_sysbios_config.o (.text.BIOS_exitFunc)
                  000078c2    0000001a     ti_sysbios_config.o (.text.ti_sysbios_knl_Semaphore_Instance_finalize)
                  000078dc    00000018     ti_sysbios_config.o (.text.BIOS_exit)
                  000078f4    00000018     drivers_cc13x2.a : GPIOCC26XX.c.obj (.text.GPIO_disableInt)
                  0000790c    00000018                      : PowerCC26X2.c.obj (.text.PowerCC26XX_calibrate)
                  00007924    00000018                      : PowerCC26X2.c.obj (.text.Power_idleFunc)
                  0000793c    00000018     rf_multiMode_cc13x2.a : RFCC26X2_multiMode.c.cc13x2.ticlang.o (.text.RF_restartClockTimeout)
                  00007954    00000018     ti_sysbios_config.o (.text.ti_sysbios_family_arm_cc26xx_Timer_getCount64)
                  0000796c    00000018     ti_sysbios_config.o (.text.ti_sysbios_family_arm_m3_Hwi_setFunc)
                  00007984    00000018     ti_sysbios_config.o (.text.ti_sysbios_knl_ClockSupport_setNextTick)
                  0000799c    00000018     sysbios.a : TaskSupport_asm_gnu.obj (.text.ti_sysbios_knl_TaskSupport_glue)
                  000079b4    00000016     ti_sysbios_config.o (.text.ClockP_Params_init)
                  000079ca    00000016     drivers_cc13x2.a : List.c.obj (.text.List_clearList)
                  000079e0    00000016     ti_sysbios_config.o (.text.ti_sysbios_family_arm_m3_Hwi_enable)
                  000079f6    00000016     ti_sysbios_config.o (.text.ti_sysbios_knl_Intrinsics_maxbit)
                  00007a0c    00000016     ti_sysbios_config.o (.text.ti_sysbios_knl_Queue_construct)
                  00007a22    00000016     ti_sysbios_config.o (.text.ti_sysbios_knl_Queue_empty)
                  00007a38    00000016     ti_sysbios_config.o (.text.ti_sysbios_runtime_System_exit)
                  00007a4e    00000014     ti_drivers_config.o (.text.Board_init)
                  00007a62    00000014     ti_sysbios_config.o (.text.ClockP_setTimeout)
                  00007a76    00000002     --HOLE-- [fill = 0]
                  00007a78    00000014     drivers_cc13x2.a : GPIOCC26XX.c.obj (.text.GPIO_toggle)
                  00007a8c    00000014     rf_multiMode_cc13x2.a : RFCC26X2_multiMode.c.cc13x2.ticlang.o (.text.RF_dbellSyncOnAck)
                  00007aa0    00000014     ti_sysbios_config.o (.text.SwiP_or)
                  00007ab4    00000014     libc.a : args_main.c.obj (.text._args_main)
                  00007ac8    00000014     ti_sysbios_config.o (.text.ti_sysbios_family_arm_cc26xx_TimestampProvider_init)
                  00007adc    00000014     ti_sysbios_config.o (.text.ti_sysbios_family_arm_m3_Hwi_disable)
                  00007af0    00000014     ti_sysbios_config.o (.text.ti_sysbios_knl_Swi_Instance_finalize)
                  00007b04    00000014     libclang_rt.builtins.a : aeabi_memset.S.obj (.text)
                  00007b18    00000014                            : aeabi_uldivmod.S.obj (.text)
                  00007b2c    00000012     ti_sysbios_config.o (.text.pthread_attr_setstacksize)
                  00007b3e    00000012     ti_sysbios_config.o (.text.ti_sysbios_family_arm_m3_Hwi_doSwiRestore)
                  00007b50    00000012     ti_sysbios_config.o (.text.ti_sysbios_family_arm_m3_Hwi_doTaskRestore)
                  00007b62    00000012     ti_sysbios_config.o (.text.ti_sysbios_heaps_HeapMem_Params_init)
                  00007b74    00000012     ti_sysbios_config.o (.text.ti_sysbios_heaps_HeapMem_init)
                  00007b86    00000012     ti_sysbios_config.o (.text.ti_sysbios_knl_Clock_Params_init)
                  00007b98    00000012     ti_sysbios_config.o (.text.ti_sysbios_knl_Clock_tick)
                  00007baa    00000012     ti_sysbios_config.o (.text.ti_sysbios_knl_Queue_Instance_init)
                  00007bbc    00000012     ti_sysbios_config.o (.text.ti_sysbios_knl_Semaphore_Params_init)
                  00007bce    00000012     libc.a : memcpy_t2.S.obj (.text:TI_memcpy_small)
                  00007be0    00000010     ti_sysbios_config.o (.text.BIOS_start)
                  00007bf0    00000010     ti_sysbios_config.o (.text.ClockP_getTimeout)
                  00007c00    00000010     ti_sysbios_config.o (.text.ClockP_isActive)
                  00007c10    00000010     ti_sysbios_config.o (.text.ClockP_start)
                  00007c20    00000010     ti_sysbios_config.o (.text.ClockP_stop)
                  00007c30    00000010     drivers_cc13x2.a : GPIOCC26XX.c.obj (.text.GPIO_write)
                  00007c40    00000010     ti_sysbios_config.o (.text.HwiP_disable)
                  00007c50    00000010     ti_sysbios_config.o (.text.HwiP_enableInterrupt)
                  00007c60    00000010     ti_sysbios_config.o (.text.HwiP_post)
                  00007c70    00000010     ti_sysbios_config.o (.text.HwiP_restore)
                  00007c80    00000010     rf_multiMode_cc13x2.a : rfc.c.cc13x2.ticlang.o (.text.NOROM_RFCCpeIntGetAndClear)
                  00007c90    00000010                           : rfc.c.cc13x2.ticlang.o (.text.NOROM_RFCHwIntGetAndClear)
                  00007ca0    00000010     drivers_cc13x2.a : PowerCC26X2_helpers.c.obj (.text.PowerCC26X2_oscCtlClearXtal)
                  00007cb0    00000010                      : PowerCC26X2_helpers.c.obj (.text.PowerCC26X2_prcmEnableCacheRetention)
                  00007cc0    00000010                      : PowerCC26X2_calibrateRCOSC_helpers.c.obj (.text.PowerCC26X2_readCtrim)
                  00007cd0    00000010                      : PowerCC26X2_calibrateRCOSC_helpers.c.obj (.text.PowerCC26X2_readCtrimFract)
                  00007ce0    00000010                      : PowerCC26X2_calibrateRCOSC_helpers.c.obj (.text.PowerCC26X2_readRtrim)
                  00007cf0    00000010                      : PowerCC26X2_helpers.c.obj (.text.PowerCC26X2_switchToTCXO)
                  00007d00    00000010     ti_sysbios_config.o (.text.SemaphoreP_post)
                  00007d10    00000010     ti_sysbios_config.o (.text.SwiP_disable)
                  00007d20    00000010     ti_sysbios_config.o (.text.SwiP_getTrigger)
                  00007d30    00000010     ti_sysbios_config.o (.text.SwiP_restore)
                  00007d40    00000010     ti_sysbios_config.o (.text.SysCtrlAonUpdate)
                  00007d50    00000010     ti_sysbios_config.o (.text.pthread_self)
                  00007d60    00000010     ti_sysbios_config.o (.text.ti_sysbios_family_arm_cc26xx_Timer_setPeriod)
                  00007d70    00000010     ti_sysbios_config.o (.text.ti_sysbios_knl_ClockSupport_getMaxTicks)
                  00007d80    00000010     ti_sysbios_config.o (.text.ti_sysbios_knl_Clock_isActive)
                  00007d90    00000010     ti_sysbios_config.o (.text.ti_sysbios_knl_Clock_removeI)
                  00007da0    00000010     ti_sysbios_config.o (.text.ti_sysbios_knl_Clock_setTimeout)
                  00007db0    00000010     ti_sysbios_config.o (.text.ti_sysbios_knl_Idle_loop)
                  00007dc0    00000010     ti_sysbios_config.o (.text.ti_sysbios_knl_Queue_destruct)
                  00007dd0    00000010     ti_sysbios_config.o (.text.ti_sysbios_knl_Queue_elemClear)
                  00007de0    00000010     ti_sysbios_config.o (.text.ti_sysbios_knl_Swi_enabled)
                  00007df0    00000010     ti_sysbios_config.o (.text.ti_sysbios_runtime_SystemSupport_exit)
                  00007e00    00000010     libc.a : copy_zero_init.c.obj (.text:decompress:ZI)
                  00007e10    0000000e     ti_sysbios_config.o (.text.BIOS_linkedWithIncorrectBootLibrary)
                  00007e1e    0000000e     ti_sysbios_config.o (.text.IntMasterDisable)
                  00007e2c    0000000e     ti_sysbios_config.o (.text.IntMasterEnable)
                  00007e3a    0000000e     drivers_cc13x2.a : PowerCC26X2.c.obj (.text.OUTLINED_FUNCTION_0)
                  00007e48    0000000e     rf_multiMode_cc13x2.a : RFCC26X2_multiMode.c.cc13x2.ticlang.o (.text.OUTLINED_FUNCTION_0)
                  00007e56    0000000e                           : RFCC26X2_multiMode.c.cc13x2.ticlang.o (.text.OUTLINED_FUNCTION_3)
                  00007e64    0000000e     drivers_cc13x2.a : PowerCC26X2.c.obj (.text.switchToTCXO)
                  00007e72    0000000e     ti_sysbios_config.o (.text.ti_sysbios_family_arm_m3_Hwi_restore)
                  00007e80    0000000e     ti_sysbios_config.o (.text.ti_sysbios_heaps_HeapMem_isBlocking)
                  00007e8e    0000000e     ti_sysbios_config.o (.text.ti_sysbios_knl_Clock_stop)
                  00007e9c    0000000e     libc.a : memset_t2.S.obj (.text:TI_memset_small)
                  00007eaa    0000000e            : copy_decompress_none.c.obj (.text:decompress:none)
                  00007eb8    0000000c     ti_sysbios_config.o (.text.AONRTCCurrentCompareValueGet)
                  00007ec4    0000000c     ti_sysbios_config.o (.text.BIOS_getThreadType)
                  00007ed0    0000000c     ti_sysbios_config.o (.text.ClockP_getSystemTickPeriod)
                  00007edc    0000000c     driverlib.lib : cpu.o (.text.NOROM_CPUcpsid)
                  00007ee8    0000000c                   : cpu.o (.text.NOROM_CPUcpsie)
                  00007ef4    0000000c     drivers_cc13x2.a : PowerCC26X2_helpers.c.obj (.text.PowerCC26X2_oscClockSourceGet)
                  00007f00    0000000c                      : PowerCC26X2_helpers.c.obj (.text.PowerCC26X2_sysCtrlGetResetSource)
                  00007f0c    0000000c                      : PowerCC26X2_helpers.c.obj (.text.PowerCC26X2_sysCtrlVoltageConditionalControl)
                  00007f18    0000000c                      : PowerCC26X2.c.obj (.text.Power_getConstraintMask)
                  00007f24    0000000c     rf_multiMode_cc13x2.a : RFCC26X2_multiMode.c.cc13x2.ticlang.o (.text.RF_Params_init)
                  00007f30    0000000c     libc.a : _lock.c.obj (.text._register_lock)
                  00007f3c    0000000c            : _lock.c.obj (.text._register_unlock)
                  00007f48    0000000c     ti_sysbios_config.o (.text.ti_sysbios_knl_Queue_head)
                  00007f54    0000000c     ti_sysbios_config.o (.text.ti_sysbios_knl_Queue_next)
                  00007f60    0000000c     ti_sysbios_config.o (.text.ti_sysbios_knl_Queue_prev)
                  00007f6c    0000000c     ti_sysbios_config.o (.text.ti_sysbios_knl_Swi_getTrigger)
                  00007f78    0000000c     ti_sysbios_config.o (.text.ti_sysbios_knl_Swi_postInit)
                  00007f84    0000000c     ti_sysbios_config.o (.text.ti_sysbios_knl_Swi_self)
                  00007f90    0000000c     ti_sysbios_config.o (.text.ti_sysbios_knl_Task_getArg1)
                  00007f9c    0000000c     ti_sysbios_config.o (.text.ti_sysbios_knl_Task_getEnv)
                  00007fa8    0000000c     ti_sysbios_config.o (.text.ti_sysbios_knl_Task_self)
                  00007fb4    0000000a     rf_multiMode_cc13x2.a : RFCC26X2_multiMode.c.cc13x2.ticlang.o (.text.OUTLINED_FUNCTION_5)
                  00007fbe    0000000a     drivers_cc13x2.a : PowerCC26X2_helpers.c.obj (.text.PowerCC26X2_sysCtrlStandby)
                  00007fc8    0000000a     ti_sysbios_config.o (.text.ti_sysbios_gates_GateMutex_handle)
                  00007fd2    0000000a     ti_sysbios_config.o (.text.ti_sysbios_knl_Clock_handle)
                  00007fdc    0000000a     ti_sysbios_config.o (.text.ti_sysbios_knl_Queue_handle)
                  00007fe6    0000000a     ti_sysbios_config.o (.text.ti_sysbios_knl_Queue_struct)
                  00007ff0    0000000a     ti_sysbios_config.o (.text.ti_sysbios_knl_Semaphore_handle)
                  00007ffa    0000000a     ti_sysbios_config.o (.text.ti_sysbios_knl_Swi_startup)
                  00008004    0000000a     ti_sysbios_config.o (.text.ti_sysbios_runtime_Error_check)
                  0000800e    0000000a     ti_sysbios_config.o (.text.ti_sysbios_runtime_Types_uargToPtr)
                  00008018    0000000a     ti_sysbios_config.o (.text.xdc_uargToPtr)
                  00008022    00000008     ti_sysbios_config.o (.text.Boot_trimDevice)
                  0000802a    00000008     driverlib.lib : cpu.o (.text.NOROM_CPUdelay)
                  00008032    00000008     rf_multiMode_cc13x2.a : RFCC26X2_multiMode.c.cc13x2.ticlang.o (.text.OUTLINED_FUNCTION_2)
                  0000803a    00000008     drivers_cc13x2.a : PowerCC26X2_helpers.c.obj (.text.PowerCC26X2_oschfTrySwitchToXosc)
                  00008042    00000008     ti_sysbios_config.o (.text.ResetISR)
                  0000804a    00000002     --HOLE-- [fill = 0]
                  0000804c    00000008     libc.a : aeabi_portable.c.obj (.text.__aeabi_errno_addr)
                  00008054    00000008     ti_sysbios_config.o (.text._system_post_cinit)
                  0000805c    00000008     ti_sysbios_config.o (.text._system_pre_init)
                  00008064    00000008     ti_sysbios_config.o (.text.ti_sysbios_family_arm_m3_Hwi_startup)
                  0000806c    00000008     ti_sysbios_config.o (.text.ti_sysbios_runtime_Startup_reset)
                  00008074    00000008     ti_sysbios_config.o (.text.ti_sysbios_runtime_SysCallback_defaultExit)
                  0000807c    00000008     ti_sysbios_config.o (.text.ti_sysbios_runtime_SystemSupport_init)
                  00008084    00000008     ti_sysbios_config.o (.text.ti_sysbios_runtime_System_exitSpin)
                  0000808c    00000006     rf_multiMode_cc13x2.a : RFCC26X2_multiMode.c.cc13x2.ticlang.o (.text.OUTLINED_FUNCTION_4)
                  00008092    00000006                           : RFCC26X2_multiMode.c.cc13x2.ticlang.o (.text.RF_clkReqAccess)
                  00008098    00000004                           : rfc.c.cc13x2.ticlang.o (.text.NOROM_RFCOverrideUpdate)
                  0000809c    00000004     ti_sysbios_config.o (.text.PRCMSleep)
                  000080a0    00000004     drivers_cc13x2.a : PowerCC26X2_helpers.c.obj (.text.PowerCC26X2_oschfSwitchToRcosc)
                  000080a4    00000004                      : PowerCC26X2_helpers.c.obj (.text.PowerCC26X2_sysCtrlIdle)
                  000080a8    00000004                      : PowerCC26X2_helpers.c.obj (.text.PowerCC26X2_turnOnXosc)
                  000080ac    00000004     rf_multiMode_cc13x2.a : RFCC26X2_multiMode.c.cc13x2.ticlang.o (.text.RF_defaultExecutionPolicy)
                  000080b0    00000004     drivers_cc13x2.a : PowerCC26X2.c.obj (.text.configureRFCoreClocks)
                  000080b4    00000004                      : PowerCC26X2.c.obj (.text.nopResourceHandler)
                  000080b8    00000004     ti_sysbios_config.o (.text.ti_sysbios_gates_GateMutex_canBlock)
                  000080bc    00000004     ti_sysbios_config.o (.text.ti_sysbios_knl_TaskSupport_getStackAlignment)
                  000080c0    00000004     ti_sysbios_config.o (.text.ti_sysbios_runtime_Memory_getMaxDefaultTypeAlign)
                  000080c4    00000004     libclang_rt.builtins.a : aeabi_memcpy.S.obj (.text)

.rodata    0    000080c8    00000e73     
                  000080c8    000005d0     ti_sysbios_config.o (.rodata.str1.1)
                  00008698    000001fc     rf_multiMode_cc13x2.a : rf_patch_cpe_prop.c.cc13x2.ticlang.o (.rodata.patchImageProp)
                  00008894    00000094     ti_sysbios_config.o (.rodata.ti_sysbios_family_arm_m3_Hwi_excHandlerMin.err)
                  00008928    0000008d     ti_sysbios_config.o (.rodata.ti_sysbios_heaps_HeapMem_alloc.err)
                  000089b5    00000089     ti_sysbios_config.o (.rodata.ti_sysbios_family_arm_m3_Hwi_Instance_init.err.1)
                  00008a3e    00000089     ti_sysbios_config.o (.rodata.ti_sysbios_family_arm_m3_Hwi_excHandlerMin.err.2)
                  00008ac7    00000089     ti_sysbios_config.o (.rodata.ti_sysbios_runtime_Memory_alloc.err)
                  00008b50    00000086     ti_sysbios_config.o (.rodata.ti_sysbios_family_arm_m3_Hwi_Instance_init.err)
                  00008bd6    00000083     ti_sysbios_config.o (.rodata.ti_sysbios_knl_Task_checkStacks.err.63)
                  00008c59    00000083     ti_sysbios_config.o (.rodata.ti_sysbios_knl_Task_checkStacks.err.64)
                  00008cdc    0000007b     ti_sysbios_config.o (.rodata.ti_sysbios_knl_Task_checkStacks.err.62)
                  00008d57    0000007b     ti_sysbios_config.o (.rodata.ti_sysbios_knl_Task_checkStacks.err)
                  00008dd2    00000054     drivers_cc13x2.a : PowerCC26X2.c.obj (.rodata.resourceDB)
                  00008e26    00000001     ti_drivers_config.o (.rodata.GPIO_pinLowerBound)
                  00008e27    00000001     ti_drivers_config.o (.rodata.GPIO_pinUpperBound)
                  00008e28    00000024     ti_sysbios_config.o (.rodata.ti_sysbios_knl_Task_Params_default)
                  00008e4c    00000020     rf_multiMode_cc13x2.a : RFCC26X2_multiMode.c.cc13x2.ticlang.o (.rodata.cst32)
                  00008e6c    0000001c     ti_sysbios_config.o (.rodata.ti_sysbios_family_arm_cc26xx_Timer_Params_default)
                  00008e88    00000018     ti_sysbios_config.o (.rodata.ti_sysbios_family_arm_m3_Hwi_Params_default)
                  00008ea0    00000014     ti_drivers_config.o (.rodata.PowerCC26X2_config)
                  00008eb4    00000014     ti_sysbios_config.o (.rodata.ti_sysbios_knl_Swi_Params_default)
                  00008ec8    00000010     ti_drivers_config.o (.rodata.GPIO_config)
                  00008ed8    0000000c     ti_drivers_config.o (.rodata.RFCC26XX_hwAttrs)
                  00008ee4    0000000c     ti_sysbios_config.o (.rodata.ti_sysbios_heaps_HeapMem_Params_default)
                  00008ef0    0000000c     ti_sysbios_config.o (.rodata.ti_sysbios_knl_Clock_Params_default)
                  00008efc    0000000c     ti_sysbios_config.o (.rodata.ti_sysbios_knl_Semaphore_Params_default)
                  00008f08    00000008     rf_multiMode_cc13x2.a : RFCC26X2_multiMode.c.cc13x2.ticlang.o (.rodata..L__const.RF_hwiCpe0Active.activeCmd)
                  00008f10    00000008     driverlib.lib : aux_sysif.o (.rodata.cst4)
                  00008f18    00000008     ti_sysbios_config.o (.rodata.ti_sysbios_knl_Idle_funcList)
                  00008f20    00000004     ti_sysbios_config.o (.rodata.ti_sysbios_family_arm_m3_Hwi_swiTaskKeyAddress)
                  00008f24    00000004     ti_sysbios_config.o (.rodata.ti_sysbios_gates_GateMutex_Params_default)
                  00008f28    00000004     ti_sysbios_config.o (.rodata.ti_sysbios_knl_Clock_tickPeriod)
                  00008f2c    00000004     ti_sysbios_config.o (.rodata.ti_sysbios_knl_Swi_numPriorities)
                  00008f30    00000004     ti_sysbios_config.o (.rodata.ti_sysbios_knl_Task_defaultStackSize)
                  00008f34    00000004     ti_sysbios_config.o (.rodata.ti_sysbios_knl_Task_numPriorities)
                  00008f38    00000001     ti_sysbios_config.o (.rodata.ti_sysbios_knl_Clock_tickMode)
                  00008f39    00000001     ti_sysbios_config.o (.rodata.ti_sysbios_knl_Task_checkStackFlag)
                  00008f3a    00000001     ti_sysbios_config.o (.rodata.ti_sysbios_knl_Task_initStackFlag)

.args      0    00008f3c    00000008     
                  00008f3c    00000008     --HOLE-- [fill = 0]

MODULE SUMMARY

       Module                                     code    ro data   rw data
       ------                                     ----    -------   -------
    .\
       rfPacketTx.o                               434     0         290    
       main_tirtos.o                              128     0         0      
    +--+------------------------------------------+-------+---------+---------+
       Total:                                     562     0         290    
                                                                           
    .\smartrf_settings\
       ti_radio_config.o                          0       0         144    
    +--+------------------------------------------+-------+---------+---------+
       Total:                                     0       0         144    
                                                                           
    .\syscfg\
       ti_sysbios_config.o                        16558   3069      1822   
       ti_drivers_config.o                        314     50        372    
       ti_devices_config.o                        0       88        0      
    +--+------------------------------------------+-------+---------+---------+
       Total:                                     16872   3207      2194   
                                                                           
    C:/ti/simplelink_cc13xx_cc26xx_sdk_6_20_00_29/kernel/tirtos7/packages/ti/sysbios/lib/ticlang/m4f/sysbios.a
       Hwi_asm_gnu.obj                            324     0         0      
       Hwi_asm_switch_gnu.obj                     118     0         0      
       TaskSupport_asm_gnu.obj                    64      0         0      
       boot_cortex_m.obj                          52      0         0      
    +--+------------------------------------------+-------+---------+---------+
       Total:                                     558     0         0      
                                                                           
    C:/ti/simplelink_cc13xx_cc26xx_sdk_6_20_00_29/source/ti/devices/cc13x2_cc26x2/driverlib/bin/ticlang/driverlib.lib
       osc.o                                      538     0         32     
       sys_ctrl.o                                 432     0         0      
       setup.o                                    392     0         0      
       chipinfo.o                                 298     0         0      
       prcm.o                                     136     0         0      
       aux_sysif.o                                72      8         0      
       cpu.o                                      32      0         0      
    +--+------------------------------------------+-------+---------+---------+
       Total:                                     1900    8         32     
                                                                           
    C:/ti/simplelink_cc13xx_cc26xx_sdk_6_20_00_29/source/ti/drivers/lib/ticlang/m4f/drivers_cc13x2.a
       PowerCC26X2.c.obj                          1790    84        372    
       PowerCC26X2_calibrateRCOSC.c.obj           836     0         0      
       PowerCC26X2_calibrateRCOSC_helpers.c.obj   436     0         0      
       GPIOCC26X2.c.obj                           328     0         29     
       PowerCC26X2_helpers.c.obj                  234     0         0      
       List.c.obj                                 208     0         0      
       GPIOCC26XX.c.obj                           200     0         0      
       GPIO.c.obj                                 60      0         0      
    +--+------------------------------------------+-------+---------+---------+
       Total:                                     4092    84        401    
                                                                           
    C:/ti/simplelink_cc13xx_cc26xx_sdk_6_20_00_29/source/ti/drivers/rf/lib/ticlang/m4f/rf_multiMode_cc13x2.a
       RFCC26X2_multiMode.c.cc13x2.ticlang.o      8044    40        1316   
       rf_patch_cpe_prop.c.cc13x2.ticlang.o       100     508       1      
       rfc.c.cc13x2.ticlang.o                     268     0         0      
    +--+------------------------------------------+-------+---------+---------+
       Total:                                     8412    548       1317   
                                                                           
    C:\ti\ti-cgt-armllvm_2.1.0.LTS\lib\armv7em-ti-none-eabihf/c/libc.a
       copy_decompress_lzss.c.obj                 106     0         0      
       autoinit.c.obj                             56      0         0      
       _lock.c.obj                                26      0         8      
       args_main.c.obj                            20      0         0      
       memcpy_t2.S.obj                            18      0         0      
       copy_zero_init.c.obj                       16      0         0      
       copy_decompress_none.c.obj                 14      0         0      
       memset_t2.S.obj                            14      0         0      
       aeabi_portable.c.obj                       8       0         4      
    +--+------------------------------------------+-------+---------+---------+
       Total:                                     278     0         12     
                                                                           
    C:\ti\ti-cgt-armllvm_2.1.0.LTS\lib\clang/14.0.5/lib/armv7em-ti-none-eabihf/libclang_rt.builtins.a
       udivmoddi4.S.obj                           176     0         0      
       aeabi_memset.S.obj                         20      0         0      
       aeabi_uldivmod.S.obj                       20      0         0      
       aeabi_memcpy.S.obj                         4       0         0      
       aeabi_div0.c.obj                           2       0         0      
    +--+------------------------------------------+-------+---------+---------+
       Total:                                     222     0         0      
                                                                           
       Stack:                                     0       0         1024   
       Linker Generated:                          0       305       0      
    +--+------------------------------------------+-------+---------+---------+
       Grand Total:                               32896   4152      5414   


LINKER GENERATED COPY TABLES

__TI_cinit_table @ 00009068 records: 2, size/record: 8, table size: 16
	.data: load addr=00008f44, load size=0000010d bytes, run addr=20004bc4, run size=00000564 bytes, compression=lzss
	.bss: load addr=00009060, load size=00000008 bytes, run addr=200040d8, run size=00000aec bytes, compression=zero_init


LINKER GENERATED HANDLER TABLE

__TI_handler_table @ 00009054 records: 3, size/record: 4, table size: 12
	index: 0, handler: __TI_decompress_lzss
	index: 1, handler: __TI_decompress_none
	index: 2, handler: __TI_zero_init


GLOBAL SYMBOLS: SORTED ALPHABETICALLY BY Name 

address   name                                                               
-------   ----                                                               
20004fb8  BIOS_Module_state                                                  
00006681  BIOS_atExitFunc                                                    
000078dd  BIOS_exit                                                          
000078a9  BIOS_exitFunc                                                      
00007ec5  BIOS_getThreadType                                                 
20004aac  BIOS_heapMemObject                                                 
00004f5f  BIOS_init                                                          
00007e11  BIOS_linkedWithIncorrectBootLibrary                                
0000096b  BIOS_nullFunc                                                      
00006d0d  BIOS_registerRTSLock                                               
00006d39  BIOS_removeRTSLock                                                 
20004ad8  BIOS_rtsGate                                                       
0000621d  BIOS_rtsLock                                                       
00006901  BIOS_rtsUnlock                                                     
000073f9  BIOS_setThreadType                                                 
00007be1  BIOS_start                                                         
00005af1  BIOS_startFunc                                                     
00007a4f  Board_init                                                         
00001363  Board_initHook                                                     
000046eb  Board_sendExtFlashByte                                             
00004fcd  Board_shutDownExtFlash                                             
000067e9  Board_wakeUpExtFlash                                               
00008023  Boot_trimDevice                                                    
000079b5  ClockP_Params_init                                                 
000055c9  ClockP_construct                                                   
00007ed1  ClockP_getSystemTickPeriod                                         
00007bf1  ClockP_getTimeout                                                  
00007c01  ClockP_isActive                                                    
00007a63  ClockP_setTimeout                                                  
00007c11  ClockP_start                                                       
00007c21  ClockP_stop                                                        
00008ec8  GPIO_config                                                        
000078f5  GPIO_disableInt                                                    
00006261  GPIO_hwiIntFxn                                                     
00002605  GPIO_init                                                          
00008e26  GPIO_pinLowerBound                                                 
00008e27  GPIO_pinUpperBound                                                 
000066bd  GPIO_resetConfig                                                   
0000409d  GPIO_setConfig                                                     
00007a79  GPIO_toggle                                                        
00007c31  GPIO_write                                                         
00004000  HEAPSIZE                                                           
00007721  HwiP_Params_init                                                   
00005735  HwiP_construct                                                     
00007c41  HwiP_disable                                                       
00007c51  HwiP_enableInterrupt                                               
00007c61  HwiP_post                                                          
00007c71  HwiP_restore                                                       
00007225  HwiP_setFunc                                                       
UNDEFED   ITM_flush                                                          
UNDEFED   ITM_restore                                                        
000079cb  List_clearList                                                     
0000741b  List_get                                                           
000070f5  List_insert                                                        
00007249  List_put                                                           
0000711b  List_putHead                                                       
00006f3d  List_remove                                                        
00005f9d  NOROM_AUXSYSIFOpModeChange                                         
00007edd  NOROM_CPUcpsid                                                     
00007ee9  NOROM_CPUcpsie                                                     
0000802b  NOROM_CPUdelay                                                     
00003a09  NOROM_ChipInfo_GetChipType                                         
00005c41  NOROM_ChipInfo_GetHwRevision                                       
000035e9  NOROM_OSCHF_AttemptToSwitchToXosc                                  
00004a4d  NOROM_OSCHF_SwitchToRcOscTurnOffXosc                               
00006e41  NOROM_OSCHF_TurnOnXosc                                             
00004ac5  NOROM_OSC_CapArrayAdjustWorkaround_Boot                            
00005dd3  NOROM_OSC_HPOSCRelativeFrequencyOffsetGet                          
000062a5  NOROM_PRCMPowerDomainsAllOff                                       
000062e9  NOROM_PRCMPowerDomainsAllOn                                        
0000550d  NOROM_RFCAnaDivTxOverride                                          
00007c81  NOROM_RFCCpeIntGetAndClear                                         
0000188b  NOROM_RFCCpePatchReset                                             
00007509  NOROM_RFCDoorbellSendTo                                            
00007c91  NOROM_RFCHwIntGetAndClear                                          
00007529  NOROM_RFCOverrideSearch                                            
00008099  NOROM_RFCOverrideUpdate                                            
00005fe5  NOROM_RFCSynthPowerDown                                            
000030b1  NOROM_SetupTrimDevice                                              
000066f9  NOROM_SysCtrlIdle                                                  
000045eb  NOROM_SysCtrlSetRechargeBeforePowerDown                            
00002905  NOROM_SysCtrlStandby                                               
00006bf9  NOROM_ThisLibraryIsFor_CC13x2_CC26x2_HwRev20AndLater_HaltIfViolated
000064c5  PowerCC26X2_RCOSC_clockFunc                                        
00001041  PowerCC26X2_auxISR                                                 
000022e5  PowerCC26X2_calibrate                                              
00008ea0  PowerCC26X2_config                                                 
00007549  PowerCC26X2_disableTCXOQual                                        
00007569  PowerCC26X2_enableTCXOQual                                         
0000531d  PowerCC26X2_initiateCalibration                                    
20004bc4  PowerCC26X2_module                                                 
00007ef5  PowerCC26X2_oscClockSourceGet                                      
00007ca1  PowerCC26X2_oscCtlClearXtal                                        
00006821  PowerCC26X2_oscDisableQualifiers                                   
000080a1  PowerCC26X2_oschfSwitchToRcosc                                     
0000803b  PowerCC26X2_oschfTrySwitchToXosc                                   
00007cb1  PowerCC26X2_prcmEnableCacheRetention                               
00007cc1  PowerCC26X2_readCtrim                                              
00007cd1  PowerCC26X2_readCtrimFract                                         
00007ce1  PowerCC26X2_readRtrim                                              
00006505  PowerCC26X2_setAclkRefSrc                                          
00006735  PowerCC26X2_setTdcClkSrc24M                                        
00007cf1  PowerCC26X2_switchToTCXO                                           
00007f01  PowerCC26X2_sysCtrlGetResetSource                                  
000080a5  PowerCC26X2_sysCtrlIdle                                            
00007fbf  PowerCC26X2_sysCtrlStandby                                         
00007f0d  PowerCC26X2_sysCtrlVoltageConditionalControl                       
000080a9  PowerCC26X2_turnOnXosc                                             
00004b3d  PowerCC26X2_updateSubSecInc                                        
0000726d  PowerCC26X2_writeCtrim                                             
00007291  PowerCC26X2_writeCtrimFract                                        
000072b5  PowerCC26X2_writeCtrimFractEn                                      
000072d9  PowerCC26X2_writeRtrim                                             
0000790d  PowerCC26XX_calibrate                                              
0000632d  PowerCC26XX_isStableXOSC_HF                                        
00007589  PowerCC26XX_schedulerDisable                                       
000075a9  PowerCC26XX_schedulerRestore                                       
0000160f  PowerCC26XX_standbyPolicy                                          
20004bb4  PowerCC26XX_swiKey                                                 
0000602d  PowerCC26XX_switchXOSC_HF                                          
20004bb8  PowerCC26XX_taskKey                                                
00007f19  Power_getConstraintMask                                            
0000773d  Power_getTransitionLatency                                         
00007925  Power_idleFunc                                                     
00001fa5  Power_init                                                         
000072fd  Power_registerNotify                                               
000069a5  Power_releaseConstraint                                            
0000369d  Power_releaseDependency                                            
00006aa9  Power_setConstraint                                                
00003751  Power_setDependency                                                
00001365  Power_sleep                                                        
00008ed8  RFCC26XX_hwAttrs                                                   
200050ec  RFCC26XX_schedulerPolicy                                           
00007f25  RF_Params_init                                                     
2000505c  RF_cmdFs                                                           
20004fe4  RF_cmdPropRadioDivSetup                                            
20005074  RF_cmdPropTx                                                       
000080ad  RF_defaultExecutionPolicy                                          
00003c99  RF_defaultSubmitPolicy                                             
00005b99  RF_getCurrentTime                                                  
000004d5  RF_open                                                            
0000395d  RF_pendCmd                                                         
00002e51  RF_postCmd                                                         
000069d9  RF_powerConstraintRelease                                          
00007791  RF_powerConstraintSet                                              
200050a0  RF_prop                                                            
00007141  RF_runCmd                                                          
00004461  RF_yield                                                           
00008043  ResetISR                                                           
00006e6b  SemaphoreP_constructBinary                                         
00006937  SemaphoreP_pend                                                    
00007d01  SemaphoreP_post                                                    
000076a9  SwiP_Params_init                                                   
00004769  SwiP_construct                                                     
00007d11  SwiP_disable                                                       
00007d21  SwiP_getTrigger                                                    
00007aa1  SwiP_or                                                            
00007d31  SwiP_restore                                                       
00007bcf  TI_memcpy_small                                                    
00007e9d  TI_memset_small                                                    
20014000  __STACK_END                                                        
00000400  __STACK_SIZE                                                       
00009068  __TI_CINIT_Base                                                    
00009078  __TI_CINIT_Limit                                                   
00009078  __TI_CINIT_Warm                                                    
00009054  __TI_Handler_Table_Base                                            
00009060  __TI_Handler_Table_Limit                                           
000068c9  __TI_auto_init_nobinit_nopinit                                     
0000517f  __TI_decompress_lzss                                               
00007eab  __TI_decompress_none                                               
ffffffff  __TI_pprof_out_hndl                                                
ffffffff  __TI_prof_data_size                                                
ffffffff  __TI_prof_data_start                                               
00000000  __TI_static_base__                                                 
00007e01  __TI_zero_init                                                     
20005110  __aeabi_errno                                                      
0000804d  __aeabi_errno_addr                                                 
000024fb  __aeabi_ldiv0                                                      
00007b11  __aeabi_memclr                                                     
00007b11  __aeabi_memclr4                                                    
00007b11  __aeabi_memclr8                                                    
000080c5  __aeabi_memcpy                                                     
000080c5  __aeabi_memcpy4                                                    
000080c5  __aeabi_memcpy8                                                    
00007b05  __aeabi_memset                                                     
00007b05  __aeabi_memset4                                                    
00007b05  __aeabi_memset8                                                    
00007b19  __aeabi_uldivmod                                                   
ffffffff  __binit__                                                          
00008f3c  __c_args__                                                         
00057fa8  __ccfg                                                             
UNDEFED   __mpu_init                                                         
200040d8  __primary_heap_end__                                               
200000d8  __primary_heap_start__                                             
20013c00  __stack                                                            
20000000  __start___llvm_prf_bits                                            
20000000  __start___llvm_prf_cnts                                            
20000000  __stop___llvm_prf_bits                                             
20000000  __stop___llvm_prf_cnts                                             
00003801  __udivmoddi4                                                       
00007ab5  _args_main                                                         
00006a75  _c_int00                                                           
200050b0  _hposcCoeffs                                                       
20005114  _lock                                                              
00002807  _nop                                                               
000063f9  _pthread_cleanupFxn                                                
00006e95  _pthread_cleanup_pop                                               
00002fe7  _pthread_removeThreadKeys                                          
00007f31  _register_lock                                                     
00007f3d  _register_unlock                                                   
00008055  _system_post_cinit                                                 
0000805d  _system_pre_init                                                   
20005118  _unlock                                                            
ffffffff  binit                                                              
20004770  gpioCallbackFunctions                                              
20004d38  gpioPinConfigs                                                     
200047ec  gpioUserArgs                                                       
0000466b  main                                                               
00000b4d  mainThread                                                         
2000500c  pOverrides                                                         
00006ebf  pthread_attr_init                                                  
00006d91  pthread_attr_setdetachstate                                        
00006605  pthread_attr_setschedparam                                         
00007b2d  pthread_attr_setstacksize                                          
000014c1  pthread_create                                                     
000047e5  pthread_exit                                                       
00007d51  pthread_self                                                       
00005bed  pthread_setcancelstate                                             
00008dd2  resourceDB                                                         
00006dbd  rf_patch_cpe_prop                                                  
200050c0  ti_sysbios_family_arm_cc26xx_Timer_Module_state                    
000073b1  ti_sysbios_family_arm_cc26xx_Timer_Params_init                     
00000ea9  ti_sysbios_family_arm_cc26xx_Timer_construct                       
000077c9  ti_sysbios_family_arm_cc26xx_Timer_dynamicStub                     
00007955  ti_sysbios_family_arm_cc26xx_Timer_getCount64                      
0000599b  ti_sysbios_family_arm_cc26xx_Timer_getCurrentTick                  
00006a0d  ti_sysbios_family_arm_cc26xx_Timer_getMaxTicks                     
00004861  ti_sysbios_family_arm_cc26xx_Timer_periodicStub                    
00007629  ti_sysbios_family_arm_cc26xx_Timer_postInit                        
00005d35  ti_sysbios_family_arm_cc26xx_Timer_setNextTick                     
00007d61  ti_sysbios_family_arm_cc26xx_Timer_setPeriod                       
00004e7d  ti_sysbios_family_arm_cc26xx_Timer_setThreshold                    
0000524f  ti_sysbios_family_arm_cc26xx_Timer_start                           
0000423f  ti_sysbios_family_arm_cc26xx_Timer_startup                         
20004bbc  ti_sysbios_family_arm_cc26xx_TimestampProvider_Module_state        
00007ac9  ti_sysbios_family_arm_cc26xx_TimestampProvider_init                
000052b5  ti_sysbios_family_arm_m3_Hwi_Instance_finalize                     
00002709  ti_sysbios_family_arm_m3_Hwi_Instance_init                         
20004f40  ti_sysbios_family_arm_m3_Hwi_Module_state                          
000077e5  ti_sysbios_family_arm_m3_Hwi_Params_init                           
000057e5  ti_sysbios_family_arm_m3_Hwi_construct                             
00004129  ti_sysbios_family_arm_m3_Hwi_construct2                            
00004c2d  ti_sysbios_family_arm_m3_Hwi_disableInterrupt                      
00001e89  ti_sysbios_family_arm_m3_Hwi_dispatch                              
00004959  ti_sysbios_family_arm_m3_Hwi_dispatchC                             
20004698  ti_sysbios_family_arm_m3_Hwi_dispatchTable                         
00007b3f  ti_sysbios_family_arm_m3_Hwi_doSwiRestore                          
00007b51  ti_sysbios_family_arm_m3_Hwi_doTaskRestore                         
00004eef  ti_sysbios_family_arm_m3_Hwi_enableInterrupt                       
00000771  ti_sysbios_family_arm_m3_Hwi_excFillContext                        
00007649  ti_sysbios_family_arm_m3_Hwi_excHandler                            
00006f8d  ti_sysbios_family_arm_m3_Hwi_excHandlerAsm                         
00003f81  ti_sysbios_family_arm_m3_Hwi_excHandlerMin                         
00007167  ti_sysbios_family_arm_m3_Hwi_getHandle                             
00004569  ti_sysbios_family_arm_m3_Hwi_getStackInfo                          
000060bd  ti_sysbios_family_arm_m3_Hwi_init                                  
00002ae7  ti_sysbios_family_arm_m3_Hwi_initNVIC                              
00006cb1  ti_sysbios_family_arm_m3_Hwi_initStack                             
0000583d  ti_sysbios_family_arm_m3_Hwi_initStacks                            
00001f60  ti_sysbios_family_arm_m3_Hwi_interruptsAreDisabledButShouldNotBe   
00001f65  ti_sysbios_family_arm_m3_Hwi_pendSV                                
00006b39  ti_sysbios_family_arm_m3_Hwi_plug                                  
00007669  ti_sysbios_family_arm_m3_Hwi_post                                  
00004351  ti_sysbios_family_arm_m3_Hwi_postInit                              
20000000  ti_sysbios_family_arm_m3_Hwi_ramVectors                            
00000000  ti_sysbios_family_arm_m3_Hwi_resetVectors                          
00001f88  ti_sysbios_family_arm_m3_Hwi_return                                
0000796d  ti_sysbios_family_arm_m3_Hwi_setFunc                               
00006771  ti_sysbios_family_arm_m3_Hwi_setPriority                           
00008065  ti_sysbios_family_arm_m3_Hwi_startup                               
00008f20  ti_sysbios_family_arm_m3_Hwi_swiTaskKeyAddress                     
000076c7  ti_sysbios_family_arm_m3_Hwi_switchAndRunFunc                      
000076e5  ti_sysbios_family_arm_m3_Hwi_switchFromBootStack                   
00006cdf  ti_sysbios_gates_GateMutex_Instance_init                           
200050f4  ti_sysbios_gates_GateMutex_Module_state                            
000080b9  ti_sysbios_gates_GateMutex_canBlock                                
00006fb5  ti_sysbios_gates_GateMutex_construct                               
00006545  ti_sysbios_gates_GateMutex_enter                                   
0000743d  ti_sysbios_gates_GateMutex_leave                                   
00003e5d  ti_sysbios_heaps_HeapMem_Instance_init                             
200050fc  ti_sysbios_heaps_HeapMem_Module_state                              
00007b63  ti_sysbios_heaps_HeapMem_Params_init                               
00005625  ti_sysbios_heaps_HeapMem_alloc                                     
0000174d  ti_sysbios_heaps_HeapMem_allocUnprotected                          
00005895  ti_sysbios_heaps_HeapMem_construct                                 
00006b69  ti_sysbios_heaps_HeapMem_free                                      
00002ca7  ti_sysbios_heaps_HeapMem_freeUnprotected                           
20004b00  ti_sysbios_heaps_HeapMem_gate                                      
00004e09  ti_sysbios_heaps_HeapMem_getStats                                  
00007b75  ti_sysbios_heaps_HeapMem_init                                      
00007e81  ti_sysbios_heaps_HeapMem_isBlocking                                
0000745f  ti_sysbios_heaps_HeapMem_restore                                   
00007689  ti_sysbios_knl_ClockSupport_getCurrentTick                         
00007d71  ti_sysbios_knl_ClockSupport_getMaxTicks                            
000054ab  ti_sysbios_knl_ClockSupport_init                                   
00007985  ti_sysbios_knl_ClockSupport_setNextTick                            
200048d0  ti_sysbios_knl_ClockSupport_timerStruct                            
000059f1  ti_sysbios_knl_Clock_Instance_init                                 
20004e1c  ti_sysbios_knl_Clock_Module_state                                  
00007b87  ti_sysbios_knl_Clock_Params_init                                   
00006b99  ti_sysbios_knl_Clock_construct                                     
00007801  ti_sysbios_knl_Clock_enqueueI                                      
00007481  ti_sysbios_knl_Clock_getTicks                                      
00006643  ti_sysbios_knl_Clock_getTicksUntilInterrupt                        
00005e6d  ti_sysbios_knl_Clock_getTimeout                                    
0000503b  ti_sysbios_knl_Clock_init                                          
00006ee9  ti_sysbios_knl_Clock_initI                                         
00007d81  ti_sysbios_knl_Clock_isActive                                      
00007d91  ti_sysbios_knl_Clock_removeI                                       
000074a3  ti_sysbios_knl_Clock_scheduleNextTick                              
00007da1  ti_sysbios_knl_Clock_setTimeout                                    
0000781d  ti_sysbios_knl_Clock_start                                         
000029f9  ti_sysbios_knl_Clock_startI                                        
00007e8f  ti_sysbios_knl_Clock_stop                                          
00007b99  ti_sysbios_knl_Clock_tick                                          
00008f38  ti_sysbios_knl_Clock_tickMode                                      
00008f28  ti_sysbios_knl_Clock_tickPeriod                                    
00003239  ti_sysbios_knl_Clock_walkQueueDynamic                              
000019c9  ti_sysbios_knl_Clock_workFuncDynamic                               
00008f18  ti_sysbios_knl_Idle_funcList                                       
000049d3  ti_sysbios_knl_Idle_init                                           
20005126  ti_sysbios_knl_Idle_initDone                                       
00007db1  ti_sysbios_knl_Idle_loop                                           
00006bc9  ti_sysbios_knl_Idle_run                                            
20004398  ti_sysbios_knl_Idle_taskStack                                      
20004930  ti_sysbios_knl_Idle_taskStruct                                     
00007bab  ti_sysbios_knl_Queue_Instance_init                                 
00007a0d  ti_sysbios_knl_Queue_construct                                     
000074c5  ti_sysbios_knl_Queue_dequeue                                       
00007dc1  ti_sysbios_knl_Queue_destruct                                      
00007dd1  ti_sysbios_knl_Queue_elemClear                                     
00007a23  ti_sysbios_knl_Queue_empty                                         
00006fdd  ti_sysbios_knl_Queue_enqueue                                       
00007f49  ti_sysbios_knl_Queue_head                                          
00007005  ti_sysbios_knl_Queue_insert                                        
00007f55  ti_sysbios_knl_Queue_next                                          
00007f61  ti_sysbios_knl_Queue_prev                                          
00006a41  ti_sysbios_knl_Queue_put                                           
00007839  ti_sysbios_knl_Queue_remove                                        
000078c3  ti_sysbios_knl_Semaphore_Instance_finalize                         
00006105  ti_sysbios_knl_Semaphore_Instance_init                             
20005104  ti_sysbios_knl_Semaphore_Module_state                              
00007bbd  ti_sysbios_knl_Semaphore_Params_init                               
00006de9  ti_sysbios_knl_Semaphore_construct                                 
000074e7  ti_sysbios_knl_Semaphore_destruct                                  
000021d5  ti_sysbios_knl_Semaphore_pend                                      
00006585  ti_sysbios_knl_Semaphore_pendTimeout                               
000041b5  ti_sysbios_knl_Semaphore_post                                      
00007af1  ti_sysbios_knl_Swi_Instance_finalize                               
00003531  ti_sysbios_knl_Swi_Instance_init                                   
20005034  ti_sysbios_knl_Swi_Module_state                                    
00007855  ti_sysbios_knl_Swi_Params_init                                     
0000614b  ti_sysbios_knl_Swi_construct                                       
0000696d  ti_sysbios_knl_Swi_construct2                                      
00007871  ti_sysbios_knl_Swi_disable                                         
00007de1  ti_sysbios_knl_Swi_enabled                                         
00007f6d  ti_sysbios_knl_Swi_getTrigger                                      
000058ed  ti_sysbios_knl_Swi_init                                            
00008f2c  ti_sysbios_knl_Swi_numPriorities                                   
0000702d  ti_sysbios_knl_Swi_or                                              
0000556b  ti_sysbios_knl_Swi_post                                            
00007f79  ti_sysbios_knl_Swi_postInit                                        
20004a4c  ti_sysbios_knl_Swi_readyQs                                         
00005d85  ti_sysbios_knl_Swi_restore                                         
000032f9  ti_sysbios_knl_Swi_restoreHwi                                      
00004ca5  ti_sysbios_knl_Swi_run                                             
0000400f  ti_sysbios_knl_Swi_runLoop                                         
000048dd  ti_sysbios_knl_Swi_schedule                                        
00007f85  ti_sysbios_knl_Swi_self                                            
00007ffb  ti_sysbios_knl_Swi_startup                                         
00000cff  ti_sysbios_knl_TaskSupport_buildTaskStack                          
00007055  ti_sysbios_knl_TaskSupport_checkStack                              
000080bd  ti_sysbios_knl_TaskSupport_getStackAlignment                       
0000799d  ti_sysbios_knl_TaskSupport_glue                                    
0000445f  ti_sysbios_knl_TaskSupport_init                                    
00003ab3  ti_sysbios_knl_TaskSupport_start                                   
0000707d  ti_sysbios_knl_TaskSupport_swap                                    
00007088  ti_sysbios_knl_TaskSupport_swapReturn                              
000023f1  ti_sysbios_knl_Task_Instance_finalize                              
000011d5  ti_sysbios_knl_Task_Instance_init                                  
20004f7c  ti_sysbios_knl_Task_Module_state                                   
000073d5  ti_sysbios_knl_Task_Params_init                                    
0000718d  ti_sysbios_knl_Task_allBlockedFunction                             
00004d1d  ti_sysbios_knl_Task_blockI                                         
00008f39  ti_sysbios_knl_Task_checkStackFlag                                 
00002bcb  ti_sysbios_knl_Task_checkStacks                                    
00005f51  ti_sysbios_knl_Task_construct                                      
00005eb9  ti_sysbios_knl_Task_create                                         
20004bc0  ti_sysbios_knl_Task_defaultStackHeap                               
00008f30  ti_sysbios_knl_Task_defaultStackSize                               
000071b3  ti_sysbios_knl_Task_delete                                         
000071d9  ti_sysbios_knl_Task_destruct                                       
0000788d  ti_sysbios_knl_Task_disable                                        
00006f13  ti_sysbios_knl_Task_enter                                          
000065c5  ti_sysbios_knl_Task_exit                                           
00007f91  ti_sysbios_knl_Task_getArg1                                        
00007f9d  ti_sysbios_knl_Task_getEnv                                         
00005681  ti_sysbios_knl_Task_init                                           
00008f3a  ti_sysbios_knl_Task_initStackFlag                                  
00008f34  ti_sysbios_knl_Task_numPriorities                                  
00003475  ti_sysbios_knl_Task_postInit                                       
00006191  ti_sysbios_knl_Task_processVitalTaskFlag                           
20004a7c  ti_sysbios_knl_Task_readyQs                                        
0000643d  ti_sysbios_knl_Task_restore                                        
000067ad  ti_sysbios_knl_Task_restoreHwi                                     
00003b55  ti_sysbios_knl_Task_schedule                                       
00007fa9  ti_sysbios_knl_Task_self                                           
00001b05  ti_sysbios_knl_Task_setPri                                         
00003ef1  ti_sysbios_knl_Task_sleep                                          
000070a5  ti_sysbios_knl_Task_sleepTimeout                                   
000044e5  ti_sysbios_knl_Task_startup                                        
00007703  ti_sysbios_knl_Task_unblock                                        
000061d7  ti_sysbios_knl_Task_unblockI                                       
00008005  ti_sysbios_runtime_Error_check                                     
200050cc  ti_sysbios_runtime_Error_ignore                                    
000071ff  ti_sysbios_runtime_Error_init                                      
00006481  ti_sysbios_runtime_Error_raiseX                                    
000043d9  ti_sysbios_runtime_Memory_alloc                                    
20005120  ti_sysbios_runtime_Memory_defaultHeapInstance                      
00006e15  ti_sysbios_runtime_Memory_free                                     
000080c1  ti_sysbios_runtime_Memory_getMaxDefaultTypeAlign                   
20005127  ti_sysbios_runtime_Startup_done                                    
00006891  ti_sysbios_runtime_Startup_exec                                    
0000806d  ti_sysbios_runtime_Startup_reset                                   
00008075  ti_sysbios_runtime_SysCallback_defaultExit                         
0000531b  ti_sysbios_runtime_SysCallback_defaultInit                         
00007df1  ti_sysbios_runtime_SystemSupport_exit                              
0000807d  ti_sysbios_runtime_SystemSupport_init                              
200050d8  ti_sysbios_runtime_System_Module_state                             
00005a47  ti_sysbios_runtime_System_atexit                                   
20004b28  ti_sysbios_runtime_System_atexitHandlers                           
00007a39  ti_sysbios_runtime_System_exit                                     
00008085  ti_sysbios_runtime_System_exitSpin                                 
000070cd  ti_sysbios_runtime_System_init                                     
00005f05  ti_sysbios_runtime_System_processAtExit                            
00005c93  usleep                                                             


GLOBAL SYMBOLS: SORTED BY Symbol Address 

address   name                                                               
-------   ----                                                               
00000000  __TI_static_base__                                                 
00000000  ti_sysbios_family_arm_m3_Hwi_resetVectors                          
00000400  __STACK_SIZE                                                       
000004d5  RF_open                                                            
00000771  ti_sysbios_family_arm_m3_Hwi_excFillContext                        
0000096b  BIOS_nullFunc                                                      
00000b4d  mainThread                                                         
00000cff  ti_sysbios_knl_TaskSupport_buildTaskStack                          
00000ea9  ti_sysbios_family_arm_cc26xx_Timer_construct                       
00001041  PowerCC26X2_auxISR                                                 
000011d5  ti_sysbios_knl_Task_Instance_init                                  
00001363  Board_initHook                                                     
00001365  Power_sleep                                                        
000014c1  pthread_create                                                     
0000160f  PowerCC26XX_standbyPolicy                                          
0000174d  ti_sysbios_heaps_HeapMem_allocUnprotected                          
0000188b  NOROM_RFCCpePatchReset                                             
000019c9  ti_sysbios_knl_Clock_workFuncDynamic                               
00001b05  ti_sysbios_knl_Task_setPri                                         
00001e89  ti_sysbios_family_arm_m3_Hwi_dispatch                              
00001f60  ti_sysbios_family_arm_m3_Hwi_interruptsAreDisabledButShouldNotBe   
00001f65  ti_sysbios_family_arm_m3_Hwi_pendSV                                
00001f88  ti_sysbios_family_arm_m3_Hwi_return                                
00001fa5  Power_init                                                         
000021d5  ti_sysbios_knl_Semaphore_pend                                      
000022e5  PowerCC26X2_calibrate                                              
000023f1  ti_sysbios_knl_Task_Instance_finalize                              
000024fb  __aeabi_ldiv0                                                      
00002605  GPIO_init                                                          
00002709  ti_sysbios_family_arm_m3_Hwi_Instance_init                         
00002807  _nop                                                               
00002905  NOROM_SysCtrlStandby                                               
000029f9  ti_sysbios_knl_Clock_startI                                        
00002ae7  ti_sysbios_family_arm_m3_Hwi_initNVIC                              
00002bcb  ti_sysbios_knl_Task_checkStacks                                    
00002ca7  ti_sysbios_heaps_HeapMem_freeUnprotected                           
00002e51  RF_postCmd                                                         
00002fe7  _pthread_removeThreadKeys                                          
000030b1  NOROM_SetupTrimDevice                                              
00003239  ti_sysbios_knl_Clock_walkQueueDynamic                              
000032f9  ti_sysbios_knl_Swi_restoreHwi                                      
00003475  ti_sysbios_knl_Task_postInit                                       
00003531  ti_sysbios_knl_Swi_Instance_init                                   
000035e9  NOROM_OSCHF_AttemptToSwitchToXosc                                  
0000369d  Power_releaseDependency                                            
00003751  Power_setDependency                                                
00003801  __udivmoddi4                                                       
0000395d  RF_pendCmd                                                         
00003a09  NOROM_ChipInfo_GetChipType                                         
00003ab3  ti_sysbios_knl_TaskSupport_start                                   
00003b55  ti_sysbios_knl_Task_schedule                                       
00003c99  RF_defaultSubmitPolicy                                             
00003e5d  ti_sysbios_heaps_HeapMem_Instance_init                             
00003ef1  ti_sysbios_knl_Task_sleep                                          
00003f81  ti_sysbios_family_arm_m3_Hwi_excHandlerMin                         
00004000  HEAPSIZE                                                           
0000400f  ti_sysbios_knl_Swi_runLoop                                         
0000409d  GPIO_setConfig                                                     
00004129  ti_sysbios_family_arm_m3_Hwi_construct2                            
000041b5  ti_sysbios_knl_Semaphore_post                                      
0000423f  ti_sysbios_family_arm_cc26xx_Timer_startup                         
00004351  ti_sysbios_family_arm_m3_Hwi_postInit                              
000043d9  ti_sysbios_runtime_Memory_alloc                                    
0000445f  ti_sysbios_knl_TaskSupport_init                                    
00004461  RF_yield                                                           
000044e5  ti_sysbios_knl_Task_startup                                        
00004569  ti_sysbios_family_arm_m3_Hwi_getStackInfo                          
000045eb  NOROM_SysCtrlSetRechargeBeforePowerDown                            
0000466b  main                                                               
000046eb  Board_sendExtFlashByte                                             
00004769  SwiP_construct                                                     
000047e5  pthread_exit                                                       
00004861  ti_sysbios_family_arm_cc26xx_Timer_periodicStub                    
000048dd  ti_sysbios_knl_Swi_schedule                                        
00004959  ti_sysbios_family_arm_m3_Hwi_dispatchC                             
000049d3  ti_sysbios_knl_Idle_init                                           
00004a4d  NOROM_OSCHF_SwitchToRcOscTurnOffXosc                               
00004ac5  NOROM_OSC_CapArrayAdjustWorkaround_Boot                            
00004b3d  PowerCC26X2_updateSubSecInc                                        
00004c2d  ti_sysbios_family_arm_m3_Hwi_disableInterrupt                      
00004ca5  ti_sysbios_knl_Swi_run                                             
00004d1d  ti_sysbios_knl_Task_blockI                                         
00004e09  ti_sysbios_heaps_HeapMem_getStats                                  
00004e7d  ti_sysbios_family_arm_cc26xx_Timer_setThreshold                    
00004eef  ti_sysbios_family_arm_m3_Hwi_enableInterrupt                       
00004f5f  BIOS_init                                                          
00004fcd  Board_shutDownExtFlash                                             
0000503b  ti_sysbios_knl_Clock_init                                          
0000517f  __TI_decompress_lzss                                               
0000524f  ti_sysbios_family_arm_cc26xx_Timer_start                           
000052b5  ti_sysbios_family_arm_m3_Hwi_Instance_finalize                     
0000531b  ti_sysbios_runtime_SysCallback_defaultInit                         
0000531d  PowerCC26X2_initiateCalibration                                    
000054ab  ti_sysbios_knl_ClockSupport_init                                   
0000550d  NOROM_RFCAnaDivTxOverride                                          
0000556b  ti_sysbios_knl_Swi_post                                            
000055c9  ClockP_construct                                                   
00005625  ti_sysbios_heaps_HeapMem_alloc                                     
00005681  ti_sysbios_knl_Task_init                                           
00005735  HwiP_construct                                                     
000057e5  ti_sysbios_family_arm_m3_Hwi_construct                             
0000583d  ti_sysbios_family_arm_m3_Hwi_initStacks                            
00005895  ti_sysbios_heaps_HeapMem_construct                                 
000058ed  ti_sysbios_knl_Swi_init                                            
0000599b  ti_sysbios_family_arm_cc26xx_Timer_getCurrentTick                  
000059f1  ti_sysbios_knl_Clock_Instance_init                                 
00005a47  ti_sysbios_runtime_System_atexit                                   
00005af1  BIOS_startFunc                                                     
00005b99  RF_getCurrentTime                                                  
00005bed  pthread_setcancelstate                                             
00005c41  NOROM_ChipInfo_GetHwRevision                                       
00005c93  usleep                                                             
00005d35  ti_sysbios_family_arm_cc26xx_Timer_setNextTick                     
00005d85  ti_sysbios_knl_Swi_restore                                         
00005dd3  NOROM_OSC_HPOSCRelativeFrequencyOffsetGet                          
00005e6d  ti_sysbios_knl_Clock_getTimeout                                    
00005eb9  ti_sysbios_knl_Task_create                                         
00005f05  ti_sysbios_runtime_System_processAtExit                            
00005f51  ti_sysbios_knl_Task_construct                                      
00005f9d  NOROM_AUXSYSIFOpModeChange                                         
00005fe5  NOROM_RFCSynthPowerDown                                            
0000602d  PowerCC26XX_switchXOSC_HF                                          
000060bd  ti_sysbios_family_arm_m3_Hwi_init                                  
00006105  ti_sysbios_knl_Semaphore_Instance_init                             
0000614b  ti_sysbios_knl_Swi_construct                                       
00006191  ti_sysbios_knl_Task_processVitalTaskFlag                           
000061d7  ti_sysbios_knl_Task_unblockI                                       
0000621d  BIOS_rtsLock                                                       
00006261  GPIO_hwiIntFxn                                                     
000062a5  NOROM_PRCMPowerDomainsAllOff                                       
000062e9  NOROM_PRCMPowerDomainsAllOn                                        
0000632d  PowerCC26XX_isStableXOSC_HF                                        
000063f9  _pthread_cleanupFxn                                                
0000643d  ti_sysbios_knl_Task_restore                                        
00006481  ti_sysbios_runtime_Error_raiseX                                    
000064c5  PowerCC26X2_RCOSC_clockFunc                                        
00006505  PowerCC26X2_setAclkRefSrc                                          
00006545  ti_sysbios_gates_GateMutex_enter                                   
00006585  ti_sysbios_knl_Semaphore_pendTimeout                               
000065c5  ti_sysbios_knl_Task_exit                                           
00006605  pthread_attr_setschedparam                                         
00006643  ti_sysbios_knl_Clock_getTicksUntilInterrupt                        
00006681  BIOS_atExitFunc                                                    
000066bd  GPIO_resetConfig                                                   
000066f9  NOROM_SysCtrlIdle                                                  
00006735  PowerCC26X2_setTdcClkSrc24M                                        
00006771  ti_sysbios_family_arm_m3_Hwi_setPriority                           
000067ad  ti_sysbios_knl_Task_restoreHwi                                     
000067e9  Board_wakeUpExtFlash                                               
00006821  PowerCC26X2_oscDisableQualifiers                                   
00006891  ti_sysbios_runtime_Startup_exec                                    
000068c9  __TI_auto_init_nobinit_nopinit                                     
00006901  BIOS_rtsUnlock                                                     
00006937  SemaphoreP_pend                                                    
0000696d  ti_sysbios_knl_Swi_construct2                                      
000069a5  Power_releaseConstraint                                            
000069d9  RF_powerConstraintRelease                                          
00006a0d  ti_sysbios_family_arm_cc26xx_Timer_getMaxTicks                     
00006a41  ti_sysbios_knl_Queue_put                                           
00006a75  _c_int00                                                           
00006aa9  Power_setConstraint                                                
00006b39  ti_sysbios_family_arm_m3_Hwi_plug                                  
00006b69  ti_sysbios_heaps_HeapMem_free                                      
00006b99  ti_sysbios_knl_Clock_construct                                     
00006bc9  ti_sysbios_knl_Idle_run                                            
00006bf9  NOROM_ThisLibraryIsFor_CC13x2_CC26x2_HwRev20AndLater_HaltIfViolated
00006cb1  ti_sysbios_family_arm_m3_Hwi_initStack                             
00006cdf  ti_sysbios_gates_GateMutex_Instance_init                           
00006d0d  BIOS_registerRTSLock                                               
00006d39  BIOS_removeRTSLock                                                 
00006d91  pthread_attr_setdetachstate                                        
00006dbd  rf_patch_cpe_prop                                                  
00006de9  ti_sysbios_knl_Semaphore_construct                                 
00006e15  ti_sysbios_runtime_Memory_free                                     
00006e41  NOROM_OSCHF_TurnOnXosc                                             
00006e6b  SemaphoreP_constructBinary                                         
00006e95  _pthread_cleanup_pop                                               
00006ebf  pthread_attr_init                                                  
00006ee9  ti_sysbios_knl_Clock_initI                                         
00006f13  ti_sysbios_knl_Task_enter                                          
00006f3d  List_remove                                                        
00006f8d  ti_sysbios_family_arm_m3_Hwi_excHandlerAsm                         
00006fb5  ti_sysbios_gates_GateMutex_construct                               
00006fdd  ti_sysbios_knl_Queue_enqueue                                       
00007005  ti_sysbios_knl_Queue_insert                                        
0000702d  ti_sysbios_knl_Swi_or                                              
00007055  ti_sysbios_knl_TaskSupport_checkStack                              
0000707d  ti_sysbios_knl_TaskSupport_swap                                    
00007088  ti_sysbios_knl_TaskSupport_swapReturn                              
000070a5  ti_sysbios_knl_Task_sleepTimeout                                   
000070cd  ti_sysbios_runtime_System_init                                     
000070f5  List_insert                                                        
0000711b  List_putHead                                                       
00007141  RF_runCmd                                                          
00007167  ti_sysbios_family_arm_m3_Hwi_getHandle                             
0000718d  ti_sysbios_knl_Task_allBlockedFunction                             
000071b3  ti_sysbios_knl_Task_delete                                         
000071d9  ti_sysbios_knl_Task_destruct                                       
000071ff  ti_sysbios_runtime_Error_init                                      
00007225  HwiP_setFunc                                                       
00007249  List_put                                                           
0000726d  PowerCC26X2_writeCtrim                                             
00007291  PowerCC26X2_writeCtrimFract                                        
000072b5  PowerCC26X2_writeCtrimFractEn                                      
000072d9  PowerCC26X2_writeRtrim                                             
000072fd  Power_registerNotify                                               
000073b1  ti_sysbios_family_arm_cc26xx_Timer_Params_init                     
000073d5  ti_sysbios_knl_Task_Params_init                                    
000073f9  BIOS_setThreadType                                                 
0000741b  List_get                                                           
0000743d  ti_sysbios_gates_GateMutex_leave                                   
0000745f  ti_sysbios_heaps_HeapMem_restore                                   
00007481  ti_sysbios_knl_Clock_getTicks                                      
000074a3  ti_sysbios_knl_Clock_scheduleNextTick                              
000074c5  ti_sysbios_knl_Queue_dequeue                                       
000074e7  ti_sysbios_knl_Semaphore_destruct                                  
00007509  NOROM_RFCDoorbellSendTo                                            
00007529  NOROM_RFCOverrideSearch                                            
00007549  PowerCC26X2_disableTCXOQual                                        
00007569  PowerCC26X2_enableTCXOQual                                         
00007589  PowerCC26XX_schedulerDisable                                       
000075a9  PowerCC26XX_schedulerRestore                                       
00007629  ti_sysbios_family_arm_cc26xx_Timer_postInit                        
00007649  ti_sysbios_family_arm_m3_Hwi_excHandler                            
00007669  ti_sysbios_family_arm_m3_Hwi_post                                  
00007689  ti_sysbios_knl_ClockSupport_getCurrentTick                         
000076a9  SwiP_Params_init                                                   
000076c7  ti_sysbios_family_arm_m3_Hwi_switchAndRunFunc                      
000076e5  ti_sysbios_family_arm_m3_Hwi_switchFromBootStack                   
00007703  ti_sysbios_knl_Task_unblock                                        
00007721  HwiP_Params_init                                                   
0000773d  Power_getTransitionLatency                                         
00007791  RF_powerConstraintSet                                              
000077c9  ti_sysbios_family_arm_cc26xx_Timer_dynamicStub                     
000077e5  ti_sysbios_family_arm_m3_Hwi_Params_init                           
00007801  ti_sysbios_knl_Clock_enqueueI                                      
0000781d  ti_sysbios_knl_Clock_start                                         
00007839  ti_sysbios_knl_Queue_remove                                        
00007855  ti_sysbios_knl_Swi_Params_init                                     
00007871  ti_sysbios_knl_Swi_disable                                         
0000788d  ti_sysbios_knl_Task_disable                                        
000078a9  BIOS_exitFunc                                                      
000078c3  ti_sysbios_knl_Semaphore_Instance_finalize                         
000078dd  BIOS_exit                                                          
000078f5  GPIO_disableInt                                                    
0000790d  PowerCC26XX_calibrate                                              
00007925  Power_idleFunc                                                     
00007955  ti_sysbios_family_arm_cc26xx_Timer_getCount64                      
0000796d  ti_sysbios_family_arm_m3_Hwi_setFunc                               
00007985  ti_sysbios_knl_ClockSupport_setNextTick                            
0000799d  ti_sysbios_knl_TaskSupport_glue                                    
000079b5  ClockP_Params_init                                                 
000079cb  List_clearList                                                     
00007a0d  ti_sysbios_knl_Queue_construct                                     
00007a23  ti_sysbios_knl_Queue_empty                                         
00007a39  ti_sysbios_runtime_System_exit                                     
00007a4f  Board_init                                                         
00007a63  ClockP_setTimeout                                                  
00007a79  GPIO_toggle                                                        
00007aa1  SwiP_or                                                            
00007ab5  _args_main                                                         
00007ac9  ti_sysbios_family_arm_cc26xx_TimestampProvider_init                
00007af1  ti_sysbios_knl_Swi_Instance_finalize                               
00007b05  __aeabi_memset                                                     
00007b05  __aeabi_memset4                                                    
00007b05  __aeabi_memset8                                                    
00007b11  __aeabi_memclr                                                     
00007b11  __aeabi_memclr4                                                    
00007b11  __aeabi_memclr8                                                    
00007b19  __aeabi_uldivmod                                                   
00007b2d  pthread_attr_setstacksize                                          
00007b3f  ti_sysbios_family_arm_m3_Hwi_doSwiRestore                          
00007b51  ti_sysbios_family_arm_m3_Hwi_doTaskRestore                         
00007b63  ti_sysbios_heaps_HeapMem_Params_init                               
00007b75  ti_sysbios_heaps_HeapMem_init                                      
00007b87  ti_sysbios_knl_Clock_Params_init                                   
00007b99  ti_sysbios_knl_Clock_tick                                          
00007bab  ti_sysbios_knl_Queue_Instance_init                                 
00007bbd  ti_sysbios_knl_Semaphore_Params_init                               
00007bcf  TI_memcpy_small                                                    
00007be1  BIOS_start                                                         
00007bf1  ClockP_getTimeout                                                  
00007c01  ClockP_isActive                                                    
00007c11  ClockP_start                                                       
00007c21  ClockP_stop                                                        
00007c31  GPIO_write                                                         
00007c41  HwiP_disable                                                       
00007c51  HwiP_enableInterrupt                                               
00007c61  HwiP_post                                                          
00007c71  HwiP_restore                                                       
00007c81  NOROM_RFCCpeIntGetAndClear                                         
00007c91  NOROM_RFCHwIntGetAndClear                                          
00007ca1  PowerCC26X2_oscCtlClearXtal                                        
00007cb1  PowerCC26X2_prcmEnableCacheRetention                               
00007cc1  PowerCC26X2_readCtrim                                              
00007cd1  PowerCC26X2_readCtrimFract                                         
00007ce1  PowerCC26X2_readRtrim                                              
00007cf1  PowerCC26X2_switchToTCXO                                           
00007d01  SemaphoreP_post                                                    
00007d11  SwiP_disable                                                       
00007d21  SwiP_getTrigger                                                    
00007d31  SwiP_restore                                                       
00007d51  pthread_self                                                       
00007d61  ti_sysbios_family_arm_cc26xx_Timer_setPeriod                       
00007d71  ti_sysbios_knl_ClockSupport_getMaxTicks                            
00007d81  ti_sysbios_knl_Clock_isActive                                      
00007d91  ti_sysbios_knl_Clock_removeI                                       
00007da1  ti_sysbios_knl_Clock_setTimeout                                    
00007db1  ti_sysbios_knl_Idle_loop                                           
00007dc1  ti_sysbios_knl_Queue_destruct                                      
00007dd1  ti_sysbios_knl_Queue_elemClear                                     
00007de1  ti_sysbios_knl_Swi_enabled                                         
00007df1  ti_sysbios_runtime_SystemSupport_exit                              
00007e01  __TI_zero_init                                                     
00007e11  BIOS_linkedWithIncorrectBootLibrary                                
00007e81  ti_sysbios_heaps_HeapMem_isBlocking                                
00007e8f  ti_sysbios_knl_Clock_stop                                          
00007e9d  TI_memset_small                                                    
00007eab  __TI_decompress_none                                               
00007ec5  BIOS_getThreadType                                                 
00007ed1  ClockP_getSystemTickPeriod                                         
00007edd  NOROM_CPUcpsid                                                     
00007ee9  NOROM_CPUcpsie                                                     
00007ef5  PowerCC26X2_oscClockSourceGet                                      
00007f01  PowerCC26X2_sysCtrlGetResetSource                                  
00007f0d  PowerCC26X2_sysCtrlVoltageConditionalControl                       
00007f19  Power_getConstraintMask                                            
00007f25  RF_Params_init                                                     
00007f31  _register_lock                                                     
00007f3d  _register_unlock                                                   
00007f49  ti_sysbios_knl_Queue_head                                          
00007f55  ti_sysbios_knl_Queue_next                                          
00007f61  ti_sysbios_knl_Queue_prev                                          
00007f6d  ti_sysbios_knl_Swi_getTrigger                                      
00007f79  ti_sysbios_knl_Swi_postInit                                        
00007f85  ti_sysbios_knl_Swi_self                                            
00007f91  ti_sysbios_knl_Task_getArg1                                        
00007f9d  ti_sysbios_knl_Task_getEnv                                         
00007fa9  ti_sysbios_knl_Task_self                                           
00007fbf  PowerCC26X2_sysCtrlStandby                                         
00007ffb  ti_sysbios_knl_Swi_startup                                         
00008005  ti_sysbios_runtime_Error_check                                     
00008023  Boot_trimDevice                                                    
0000802b  NOROM_CPUdelay                                                     
0000803b  PowerCC26X2_oschfTrySwitchToXosc                                   
00008043  ResetISR                                                           
0000804d  __aeabi_errno_addr                                                 
00008055  _system_post_cinit                                                 
0000805d  _system_pre_init                                                   
00008065  ti_sysbios_family_arm_m3_Hwi_startup                               
0000806d  ti_sysbios_runtime_Startup_reset                                   
00008075  ti_sysbios_runtime_SysCallback_defaultExit                         
0000807d  ti_sysbios_runtime_SystemSupport_init                              
00008085  ti_sysbios_runtime_System_exitSpin                                 
00008099  NOROM_RFCOverrideUpdate                                            
000080a1  PowerCC26X2_oschfSwitchToRcosc                                     
000080a5  PowerCC26X2_sysCtrlIdle                                            
000080a9  PowerCC26X2_turnOnXosc                                             
000080ad  RF_defaultExecutionPolicy                                          
000080b9  ti_sysbios_gates_GateMutex_canBlock                                
000080bd  ti_sysbios_knl_TaskSupport_getStackAlignment                       
000080c1  ti_sysbios_runtime_Memory_getMaxDefaultTypeAlign                   
000080c5  __aeabi_memcpy                                                     
000080c5  __aeabi_memcpy4                                                    
000080c5  __aeabi_memcpy8                                                    
00008dd2  resourceDB                                                         
00008e26  GPIO_pinLowerBound                                                 
00008e27  GPIO_pinUpperBound                                                 
00008ea0  PowerCC26X2_config                                                 
00008ec8  GPIO_config                                                        
00008ed8  RFCC26XX_hwAttrs                                                   
00008f18  ti_sysbios_knl_Idle_funcList                                       
00008f20  ti_sysbios_family_arm_m3_Hwi_swiTaskKeyAddress                     
00008f28  ti_sysbios_knl_Clock_tickPeriod                                    
00008f2c  ti_sysbios_knl_Swi_numPriorities                                   
00008f30  ti_sysbios_knl_Task_defaultStackSize                               
00008f34  ti_sysbios_knl_Task_numPriorities                                  
00008f38  ti_sysbios_knl_Clock_tickMode                                      
00008f39  ti_sysbios_knl_Task_checkStackFlag                                 
00008f3a  ti_sysbios_knl_Task_initStackFlag                                  
00008f3c  __c_args__                                                         
00009054  __TI_Handler_Table_Base                                            
00009060  __TI_Handler_Table_Limit                                           
00009068  __TI_CINIT_Base                                                    
00009078  __TI_CINIT_Limit                                                   
00009078  __TI_CINIT_Warm                                                    
00057fa8  __ccfg                                                             
20000000  __start___llvm_prf_bits                                            
20000000  __start___llvm_prf_cnts                                            
20000000  __stop___llvm_prf_bits                                             
20000000  __stop___llvm_prf_cnts                                             
20000000  ti_sysbios_family_arm_m3_Hwi_ramVectors                            
200000d8  __primary_heap_start__                                             
200040d8  __primary_heap_end__                                               
20004398  ti_sysbios_knl_Idle_taskStack                                      
20004698  ti_sysbios_family_arm_m3_Hwi_dispatchTable                         
20004770  gpioCallbackFunctions                                              
200047ec  gpioUserArgs                                                       
200048d0  ti_sysbios_knl_ClockSupport_timerStruct                            
20004930  ti_sysbios_knl_Idle_taskStruct                                     
20004a4c  ti_sysbios_knl_Swi_readyQs                                         
20004a7c  ti_sysbios_knl_Task_readyQs                                        
20004aac  BIOS_heapMemObject                                                 
20004ad8  BIOS_rtsGate                                                       
20004b00  ti_sysbios_heaps_HeapMem_gate                                      
20004b28  ti_sysbios_runtime_System_atexitHandlers                           
20004bb4  PowerCC26XX_swiKey                                                 
20004bb8  PowerCC26XX_taskKey                                                
20004bbc  ti_sysbios_family_arm_cc26xx_TimestampProvider_Module_state        
20004bc0  ti_sysbios_knl_Task_defaultStackHeap                               
20004bc4  PowerCC26X2_module                                                 
20004d38  gpioPinConfigs                                                     
20004e1c  ti_sysbios_knl_Clock_Module_state                                  
20004f40  ti_sysbios_family_arm_m3_Hwi_Module_state                          
20004f7c  ti_sysbios_knl_Task_Module_state                                   
20004fb8  BIOS_Module_state                                                  
20004fe4  RF_cmdPropRadioDivSetup                                            
2000500c  pOverrides                                                         
20005034  ti_sysbios_knl_Swi_Module_state                                    
2000505c  RF_cmdFs                                                           
20005074  RF_cmdPropTx                                                       
200050a0  RF_prop                                                            
200050b0  _hposcCoeffs                                                       
200050c0  ti_sysbios_family_arm_cc26xx_Timer_Module_state                    
200050cc  ti_sysbios_runtime_Error_ignore                                    
200050d8  ti_sysbios_runtime_System_Module_state                             
200050ec  RFCC26XX_schedulerPolicy                                           
200050f4  ti_sysbios_gates_GateMutex_Module_state                            
200050fc  ti_sysbios_heaps_HeapMem_Module_state                              
20005104  ti_sysbios_knl_Semaphore_Module_state                              
20005110  __aeabi_errno                                                      
20005114  _lock                                                              
20005118  _unlock                                                            
20005120  ti_sysbios_runtime_Memory_defaultHeapInstance                      
20005126  ti_sysbios_knl_Idle_initDone                                       
20005127  ti_sysbios_runtime_Startup_done                                    
20013c00  __stack                                                            
20014000  __STACK_END                                                        
ffffffff  __TI_pprof_out_hndl                                                
ffffffff  __TI_prof_data_size                                                
ffffffff  __TI_prof_data_start                                               
ffffffff  __binit__                                                          
ffffffff  binit                                                              
UNDEFED   ITM_flush                                                          
UNDEFED   ITM_restore                                                        
UNDEFED   __mpu_init                                                         

[446 symbols]
